Component: ARM Compiler 5.06 update 7 (build 960) Tool: armlink [4d3601]

==============================================================================

Section Cross References

    startup_rtl876x.o(VECTOR) refers to startup_rtl876x.o(RESET) for Reset_Handler
    startup_rtl876x.o(VECTOR) refers to startup_rtl876x.o(.text) for NMI_Handler
    startup_rtl876x.o(VECTOR) refers to main.o(.app.data_ram.text) for System_Handler
    startup_rtl876x.o(VECTOR) refers to rcu_dtm_app.o(.text) for UART0_Handler
    startup_rtl876x.o(VECTOR) refers to rtc_driver.o(.app.data_ram.text) for RTC_Handler
    startup_rtl876x.o(VECTOR) refers to voice_driver.o(.app.data_ram.text) for GDMA0_Channel0_Handler
    startup_rtl876x.o(VECTOR) refers to ir_send_driver.o(.app.data_ram.text) for GDMA0_Channel1_Handler
    startup_rtl876x.o(VECTOR) refers to system_rtl876x.o(.app.data_ram.text) for GPIO_Group3_Handler
    startup_rtl876x.o(VECTOR) refers to reset_watch_dog_timer.o(.app.data_ram.text) for Timer5_Handler
    startup_rtl876x.o(VECTOR) refers to keyscan_driver.o(.app.data_ram.text) for Keyscan_Handler
    startup_rtl876x.o(RESET) refers to system_rtl876x.o(.app.flash.text) for SystemInit
    system_rtl876x.o(.app.data_ram.text) refers to startup_rtl876x.o(.text) for GPIO3_Handler
    system_rtl876x.o(.app.flash.text) refers to overlay_mgr.o(.text) for load_overlay
    system_rtl876x.o(.app.flash.text) refers to system_rtl876x.o(.app.overlay_a) for AppUpdateVectorTable
    system_rtl876x.o(.app.flash.text) refers to system_rtl876x.o(.bss) for user_wdg_cb
    system_rtl876x.o(.app.flash.text) refers to system_rtl876x.o(.TRACE) for .TRACE
    system_rtl876x.o(.app.flash.text) refers to main.o(.data) for app_pre_main_cb
    system_rtl876x.o(.app.flash.text) refers to system_rtl876x.o(.text) for common_main
==============================================================================

Removing Unused input sections from the image.

    Removing system_rtl876x.o(.rev16_text), (4 bytes).
    Removing system_rtl876x.o(.revsh_text), (4 bytes).
    Removing rtl876x_io_dlps.o(.rev16_text), (4 bytes).
    Removing rtl876x_io_dlps.o(.revsh_text), (4 bytes).
    Removing rtl876x_gpio.o(.rev16_text), (4 bytes).
    Removing rtl876x_gpio.o(.revsh_text), (4 bytes).
    Removing rtl876x_ir.o(.rev16_text), (4 bytes).
    Removing rtl876x_ir.o(.revsh_text), (4 bytes).
    Removing rtl876x_keyscan.o(.rev16_text), (4 bytes).
    Removing rtl876x_keyscan.o(.revsh_text), (4 bytes).
    Removing rtl876x_rtc.o(.rev16_text), (4 bytes).
    Removing rtl876x_rtc.o(.revsh_text), (4 bytes).
    Removing rtl876x_codec.o(.rev16_text), (4 bytes).
    Removing rtl876x_codec.o(.revsh_text), (4 bytes).
    Removing rtl876x_i2s.o(.rev16_text), (4 bytes).
    Removing rtl876x_i2s.o(.revsh_text), (4 bytes).
    Removing rtl876x_pinmux.o(.rev16_text), (4 bytes).
    Removing rtl876x_pinmux.o(.revsh_text), (4 bytes).
==============================================================================

Image Symbol Table

    Local Symbols

    Symbol Name                              Value     Ov Type        Size  Object(Section)

    ../clib/angel/boardlib.s                 0x00000000   Number         0  boardinit2.o ABSOLUTE
    ../clib/angel/boardlib.s                 0x00000000   Number         0  boardinit3.o ABSOLUTE
    ../clib/angel/boardlib.s                 0x00000000   Number         0  boardinit1.o ABSOLUTE
    ../clib/angel/kernel.s                   0x00000000   Number         0  __rtentry4.o ABSOLUTE
    ../clib/angel/kernel.s                   0x00000000   Number         0  __rtentry.o ABSOLUTE
    ../clib/angel/kernel.s                   0x00000000   Number         0  __rtentry2.o ABSOLUTE
    ../clib/angel/kernel.s                   0x00000000   Number         0  __rtentry5.o ABSOLUTE
    ../clib/angel/rt.s                       0x00000000   Number         0  aeabi_idiv0.o ABSOLUTE
    ../clib/angel/rt.s                       0x00000000   Number         0  rt_ctype_table.o ABSOLUTE
    ../clib/angel/rt.s                       0x00000000   Number         0  rt_locale_intlibspace.o ABSOLUTE
    ../clib/angel/rt.s                       0x00000000   Number         0  rt_raise.o ABSOLUTE
    ../clib/angel/rt.s                       0x00000000   Number         0  rt_locale.o ABSOLUTE
    ../clib/angel/rt.s                       0x00000000   Number         0  aeabi_ldiv0_sigfpe.o ABSOLUTE
    ../clib/angel/rt.s                       0x00000000   Number         0  aeabi_ldiv0.o ABSOLUTE
    ../clib/angel/rt.s                       0x00000000   Number         0  aeabi_idiv0_sigfpe.o ABSOLUTE
    ../clib/angel/rt.s                       0x00000000   Number         0  rt_div0.o ABSOLUTE
    ../clib/angel/startup.s                  0x00000000   Number         0  __main.o ABSOLUTE
    ../clib/angel/sys.s                      0x00000000   Number         0  indicate_semi.o ABSOLUTE
    ../clib/angel/sys.s                      0x00000000   Number         0  use_no_semi.o ABSOLUTE
    ../clib/angel/sys.s                      0x00000000   Number         0  libspace.o ABSOLUTE
    ../clib/angel/sysapp.c                   0x00000000   Number         0  sys_exit.o ABSOLUTE
    ../clib/angel/sysapp.c                   0x00000000   Number         0  sys_command.o ABSOLUTE
    ../clib/angel/sysapp.c                   0x00000000   Number         0  sys_wrch.o ABSOLUTE
    ../clib/armsys.c                         0x00000000   Number         0  no_argv.o ABSOLUTE
    ../clib/armsys.c                         0x00000000   Number         0  _get_argv_nomalloc.o ABSOLUTE
    ../clib/armsys.c                         0x00000000   Number         0  argv_veneer.o ABSOLUTE
    ../clib/bigflt.c                         0x00000000   Number         0  bigflt0.o ABSOLUTE
    ../clib/btod.c                           0x00000000   Number         0  btod.o ABSOLUTE
    ../clib/division.c                       0x00000000   Number         0  lludiv.o ABSOLUTE
    ../clib/division.c                       0x00000000   Number         0  rtudiv10.o ABSOLUTE
    ../clib/division.c                       0x00000000   Number         0  lludiv10.o ABSOLUTE
    ../clib/division.s                       0x00000000   Number         0  aeabi_sdiv_div0.o ABSOLUTE
    ../clib/division.s                       0x00000000   Number         0  aeabi_sdiv.o ABSOLUTE
    ../clib/heapalloc.c                      0x00000000   Number         0  hrguard.o ABSOLUTE
    ../clib/libinit.s                        0x00000000   Number         0  libinit2.o ABSOLUTE
    ../clib/libinit.s                        0x00000000   Number         0  libinit.o ABSOLUTE
    ../clib/locale.c                         0x00000000   Number         0  _wcrtomb.o ABSOLUTE
    ../clib/locale.s                         0x00000000   Number         0  lc_ctype_c.o ABSOLUTE
    ../clib/locale.s                         0x00000000   Number         0  lc_numeric_c.o ABSOLUTE
    ../clib/longlong.c                       0x00000000   Number         0  llmul.o ABSOLUTE
    ../clib/misc.s                           0x00000000   Number         0  printf_stubs.o ABSOLUTE
    ../clib/printf.c                         0x00000000   Number         0  _printf_char.o ABSOLUTE
    ../clib/printf.c                         0x00000000   Number         0  _printf_wchar.o ABSOLUTE
    ../clib/printf.c                         0x00000000   Number         0  _printf_hex_int_ll.o ABSOLUTE
    ../clib/printf.c                         0x00000000   Number         0  _printf_fp_infnan.o ABSOLUTE
    ../clib/printf.c                         0x00000000   Number         0  vsprintf.o ABSOLUTE
    ../clib/printf.c                         0x00000000   Number         0  _printf_hex_ptr.o ABSOLUTE
    ../clib/printf.c                         0x00000000   Number         0  _printf_hex_int.o ABSOLUTE
    ../clib/printf.c                         0x00000000   Number         0  __printf_flags_ss_wp.o ABSOLUTE
    ../clib/printf.c                         0x00000000   Number         0  __printf_ss_wp.o ABSOLUTE
    ../clib/printf.c                         0x00000000   Number         0  __printf_flags_wp.o ABSOLUTE
    ../clib/printf.c                         0x00000000   Number         0  __printf_wp.o ABSOLUTE
    ../clib/printf.c                         0x00000000   Number         0  __printf_flags_ss.o ABSOLUTE
    ../clib/printf.c                         0x00000000   Number         0  __printf_ss.o ABSOLUTE
    ../clib/printf.c                         0x00000000   Number         0  __printf_flags.o ABSOLUTE
    ../clib/printf.c                         0x00000000   Number         0  _printf_hex_int_ll_ptr.o ABSOLUTE
    ../clib/printf.c                         0x00000000   Number         0  _printf_hex_ll_ptr.o ABSOLUTE
    ../clib/printf.c                         0x00000000   Number         0  __printf.o ABSOLUTE
    ../clib/printf.c                         0x00000000   Number         0  _printf_hex_int_ptr.o ABSOLUTE
    ../clib/printf.c                         0x00000000   Number         0  _printf_pad.o ABSOLUTE
    ../clib/printf.c                         0x00000000   Number         0  _printf_truncate.o ABSOLUTE
    ../clib/printf.c                         0x00000000   Number         0  _printf_str.o ABSOLUTE
    ../clib/printf.c                         0x00000000   Number         0  _printf_dec.o ABSOLUTE
    ../clib/printf.c                         0x00000000   Number         0  _printf_charcount.o ABSOLUTE
    ../clib/printf.c                         0x00000000   Number         0  _printf_char_common.o ABSOLUTE
    ../clib/printf.c                         0x00000000   Number         0  _sputc.o ABSOLUTE
    ../clib/printf.c                         0x00000000   Number         0  _printf_wctomb.o ABSOLUTE
    ../clib/printf.c                         0x00000000   Number         0  _printf_longlong_dec.o ABSOLUTE
    ../clib/printf.c                         0x00000000   Number         0  _printf_oct_ll.o ABSOLUTE
    ../clib/printf.c                         0x00000000   Number         0  _printf_oct_int.o ABSOLUTE
    ../clib/printf.c                         0x00000000   Number         0  _printf_hex_ll.o ABSOLUTE
    ../clib/printf.c                         0x00000000   Number         0  _printf_oct_int_ll.o ABSOLUTE
    ../clib/printf.c                         0x00000000   Number         0  _printf_fp_dec.o ABSOLUTE
    ../clib/printf.c                         0x00000000   Number         0  _printf_fp_hex.o ABSOLUTE
    ../clib/printf.c                         0x00000000   Number         0  __printf_nopercent.o ABSOLUTE
    ../clib/printf.c                         0x00000000   Number         0  _printf_intcommon.o ABSOLUTE
    ../clib/printf_percent.s                 0x00000000   Number         0  _printf_f.o ABSOLUTE
    ../clib/printf_percent.s                 0x00000000   Number         0  _printf_u.o ABSOLUTE
    ../clib/printf_percent.s                 0x00000000   Number         0  _printf_lld.o ABSOLUTE
    ../clib/printf_percent.s                 0x00000000   Number         0  _printf_n.o ABSOLUTE
    ../clib/printf_percent.s                 0x00000000   Number         0  _printf_e.o ABSOLUTE
    ../clib/printf_percent.s                 0x00000000   Number         0  _printf_llu.o ABSOLUTE
    ../clib/printf_percent.s                 0x00000000   Number         0  _printf_g.o ABSOLUTE
    ../clib/printf_percent.s                 0x00000000   Number         0  _printf_a.o ABSOLUTE
    ../clib/printf_percent.s                 0x00000000   Number         0  _printf_ll.o ABSOLUTE
    ../clib/printf_percent.s                 0x00000000   Number         0  _printf_percent_end.o ABSOLUTE
    ../clib/printf_percent.s                 0x00000000   Number         0  _printf_x.o ABSOLUTE
    ../clib/printf_percent.s                 0x00000000   Number         0  _printf_percent.o ABSOLUTE
    ../clib/printf_percent.s                 0x00000000   Number         0  _printf_p.o ABSOLUTE
    ../clib/printf_percent.s                 0x00000000   Number         0  _printf_c.o ABSOLUTE
    ../clib/printf_percent.s                 0x00000000   Number         0  _printf_llx.o ABSOLUTE
    ../clib/printf_percent.s                 0x00000000   Number         0  _printf_l.o ABSOLUTE
    ../clib/printf_percent.s                 0x00000000   Number         0  _printf_lc.o ABSOLUTE
    ../clib/printf_percent.s                 0x00000000   Number         0  _printf_ls.o ABSOLUTE
    ../clib/printf_percent.s                 0x00000000   Number         0  _printf_llo.o ABSOLUTE
    ../clib/printf_percent.s                 0x00000000   Number         0  _printf_o.o ABSOLUTE
    ../clib/printf_percent.s                 0x00000000   Number         0  _printf_d.o ABSOLUTE
    ../clib/printf_percent.s                 0x00000000   Number         0  _printf_s.o ABSOLUTE
    ../clib/printf_percent.s                 0x00000000   Number         0  _printf_lli.o ABSOLUTE
    ../clib/printf_percent.s                 0x00000000   Number         0  _printf_i.o ABSOLUTE
    ../clib/signal.c                         0x00000000   Number         0  defsig_abrt_inner.o ABSOLUTE
    ../clib/signal.c                         0x00000000   Number         0  defsig_rtred_inner.o ABSOLUTE
    ../clib/signal.c                         0x00000000   Number         0  defsig_stak_inner.o ABSOLUTE
    ../clib/signal.c                         0x00000000   Number         0  defsig_fpe_outer.o ABSOLUTE
    ../clib/signal.c                         0x00000000   Number         0  defsig_fpe_formal.o ABSOLUTE
    ../clib/signal.c                         0x00000000   Number         0  defsig_exit.o ABSOLUTE
    ../clib/signal.c                         0x00000000   Number         0  defsig_pvfn_inner.o ABSOLUTE
    ../clib/signal.c                         0x00000000   Number         0  defsig_fpe_inner.o ABSOLUTE
    ../clib/signal.c                         0x00000000   Number         0  defsig_cppl_inner.o ABSOLUTE
    ../clib/signal.c                         0x00000000   Number         0  defsig_rtmem_outer.o ABSOLUTE
    ../clib/signal.c                         0x00000000   Number         0  defsig_segv_inner.o ABSOLUTE
    ../clib/signal.c                         0x00000000   Number         0  defsig_rtmem_formal.o ABSOLUTE
    ../clib/signal.c                         0x00000000   Number         0  __raise.o ABSOLUTE
    ../clib/signal.c                         0x00000000   Number         0  defsig_general.o ABSOLUTE
    ../clib/signal.c                         0x00000000   Number         0  defsig_rtmem_inner.o ABSOLUTE
    ../clib/signal.c                         0x00000000   Number         0  defsig_other.o ABSOLUTE
    ../clib/signal.s                         0x00000000   Number         0  defsig.o ABSOLUTE
    ../clib/stdlib.c                         0x00000000   Number         0  rand.o ABSOLUTE
    ../clib/stdlib.c                         0x00000000   Number         0  rand.o ABSOLUTE
    ../clib/string.c                         0x00000000   Number         0  strcmp.o ABSOLUTE
    ../fplib/cfplib/d2f.c                    0x00000000   Number         0  d2f.o ABSOLUTE
    ../fplib/cfplib/daddsub.c                0x00000000   Number         0  daddsub.o ABSOLUTE
    ../fplib/cfplib/ddiv.c                   0x00000000   Number         0  ddiv.o ABSOLUTE
    ../fplib/cfplib/dmul.c                   0x00000000   Number         0  dmul.o ABSOLUTE
    ../fplib/cfplib/f2d.c                    0x00000000   Number         0  f2d.o ABSOLUTE
    ../fplib/cfplib/fdiv.c                   0x00000000   Number         0  fdiv.o ABSOLUTE
    ../fplib/cfplib/ffix.c                   0x00000000   Number         0  dfixui.o ABSOLUTE
    ../fplib/cfplib/ffix.c                   0x00000000   Number         0  ffixui.o ABSOLUTE
    ../fplib/cfplib/fflt.c                   0x00000000   Number         0  dflti.o ABSOLUTE
    ../fplib/cfplib/fflt.c                   0x00000000   Number         0  fflti.o ABSOLUTE
    ../fplib/cfplib/fpinit.c                 0x00000000   Number         0  fpinit.o ABSOLUTE
    ../fplib/cfplib/ieee_status.c            0x00000000   Number         0  ieee_status.o ABSOLUTE
    ../fplib/faddsub6m.s                     0x00000000   Number         0  faddsub.o ABSOLUTE
    ../fplib/fmul6m.s                        0x00000000   Number         0  fmul.o ABSOLUTE
    ../fplib/printf1.s                       0x00000000   Number         0  printf1.o ABSOLUTE
    ../fplib/printf2.s                       0x00000000   Number         0  printf2.o ABSOLUTE
    ../fplib/printf2a.s                      0x00000000   Number         0  printf2a.o ABSOLUTE
    ../fplib/printf2b.s                      0x00000000   Number         0  printf2b.o ABSOLUTE
    ../fplib/usenofp.s                       0x00000000   Number         0  usenofp.o ABSOLUTE
    ../mathlib/fpclassify.c                  0x00000000   Number         0  fpclassify.o ABSOLUTE
    ..\..\..\..\src\app\adc_lib\adc_lib.c    0x00000000   Number         0  adc_lib.o ABSOLUTE
    ..\..\..\..\src\app\gap_lib\systemcall\gap_lib_system_call.c 0x00000000   Number         0  gap_lib_system_call.o ABSOLUTE
    ..\..\..\..\src\app\google_rcu\address_module\rcu_link_mgr.c 0x00000000   Number         0  rcu_link_mgr.o ABSOLUTE
    ..\..\..\..\src\app\google_rcu\app_task.c 0x00000000   Number         0  app_task.o ABSOLUTE
    ..\..\..\..\src\app\google_rcu\bat_module\battery_driver.c 0x00000000   Number         0  battery_driver.o ABSOLUTE
    ..\..\..\..\src\app\google_rcu\buzzer_module\buzzer_driver.c 0x00000000   Number         0  buzzer_driver.o ABSOLUTE
    ..\..\..\..\src\app\google_rcu\buzzer_module\fms_service_handle.c 0x00000000   Number         0  fms_service_handle.o ABSOLUTE
    ..\..\..\..\src\app\google_rcu\dtm_module\rcu_dtm_app.c 0x00000000   Number         0  rcu_dtm_app.o ABSOLUTE
    ..\..\..\..\src\app\google_rcu\frm_vpk\frm_vpk_api\frm_vpk_hal_sflash.c 0x00000000   Number         0  frm_vpk_hal_sflash.o ABSOLUTE
    ..\..\..\..\src\app\google_rcu\frm_vpk\frm_vpk_api\frm_vpk_log.c 0x00000000   Number         0  frm_vpk_log.o ABSOLUTE
    ..\..\..\..\src\app\google_rcu\frm_vpk\src\app_custom.c 0x00000000   Number         0  app_custom.o ABSOLUTE
    ..\..\..\..\src\app\google_rcu\frm_vpk\src\app_flash_write.c 0x00000000   Number         0  app_flash_write.o ABSOLUTE
    ..\..\..\..\src\app\google_rcu\ir_module\ir_protocol_nec.c 0x00000000   Number         0  ir_protocol_nec.o ABSOLUTE
    ..\..\..\..\src\app\google_rcu\ir_module\ir_send_driver.c 0x00000000   Number         0  ir_send_driver.o ABSOLUTE
    ..\..\..\..\src\app\google_rcu\ir_module\ir_send_handle.c 0x00000000   Number         0  ir_send_handle.o ABSOLUTE
    ..\..\..\..\src\app\google_rcu\ir_module\ir_service_handle.c 0x00000000   Number         0  ir_service_handle.o ABSOLUTE
    ..\..\..\..\src\app\google_rcu\key_module\key_handle.c 0x00000000   Number         0  key_handle.o ABSOLUTE
    ..\..\..\..\src\app\google_rcu\key_module\keyscan_driver.c 0x00000000   Number         0  keyscan_driver.o ABSOLUTE
    ..\..\..\..\src\app\google_rcu\led_module\led_driver.c 0x00000000   Number         0  led_driver.o ABSOLUTE
    ..\..\..\..\src\app\google_rcu\led_module\led_pwm_driver.c 0x00000000   Number         0  led_pwm_driver.o ABSOLUTE
    ..\..\..\..\src\app\google_rcu\loop_queue.c 0x00000000   Number         0  loop_queue.o ABSOLUTE
    ..\..\..\..\src\app\google_rcu\main.c    0x00000000   Number         0  main.o ABSOLUTE
    ..\..\..\..\src\app\google_rcu\profile_module\dfu_service.c 0x00000000   Number         0  dfu_service.o ABSOLUTE
    ..\..\..\..\src\app\google_rcu\profile_module\fms.c 0x00000000   Number         0  fms.o ABSOLUTE
    ..\..\..\..\src\app\google_rcu\profile_module\hids_rmc.c 0x00000000   Number         0  hids_rmc.o ABSOLUTE
    ..\..\..\..\src\app\google_rcu\profile_module\ir_service.c 0x00000000   Number         0  ir_service.o ABSOLUTE
    ..\..\..\..\src\app\google_rcu\profile_module\ota_service.c 0x00000000   Number         0  ota_service.o ABSOLUTE
    ..\..\..\..\src\app\google_rcu\rcu_application.c 0x00000000   Number         0  rcu_application.o ABSOLUTE
    ..\..\..\..\src\app\google_rcu\rcu_gap.c 0x00000000   Number         0  rcu_gap.o ABSOLUTE
    ..\..\..\..\src\app\google_rcu\reset_watch_dog_timer.c 0x00000000   Number         0  reset_watch_dog_timer.o ABSOLUTE
    ..\..\..\..\src\app\google_rcu\rtc_module\rtc_driver.c 0x00000000   Number         0  rtc_driver.o ABSOLUTE
    ..\..\..\..\src\app\google_rcu\swtimer.c 0x00000000   Number         0  swtimer.o ABSOLUTE
    ..\..\..\..\src\app\google_rcu\test_module\data_uart_test.c 0x00000000   Number         0  data_uart_test.o ABSOLUTE
    ..\..\..\..\src\app\google_rcu\test_module\mp_test.c 0x00000000   Number         0  mp_test.o ABSOLUTE
    ..\..\..\..\src\app\google_rcu\test_module\single_tone.c 0x00000000   Number         0  single_tone.o ABSOLUTE
    ..\..\..\..\src\app\google_rcu\test_module\uart_transport.c 0x00000000   Number         0  uart_transport.o ABSOLUTE
    ..\..\..\..\src\app\google_rcu\voice_module\voice.c 0x00000000   Number         0  voice.o ABSOLUTE
    ..\..\..\..\src\app\google_rcu\voice_module\voice_driver.c 0x00000000   Number         0  voice_driver.o ABSOLUTE
    ..\..\..\..\src\ble\privacy\privacy_mgnt.c 0x00000000   Number         0  privacy_mgnt.o ABSOLUTE
    ..\..\..\..\src\ble\profile\server\atvv_service.c 0x00000000   Number         0  atvv_service.o ABSOLUTE
    ..\..\..\..\src\ble\profile\server\bas.c 0x00000000   Number         0  bas.o ABSOLUTE
    ..\..\..\..\src\ble\profile\server\dis.c 0x00000000   Number         0  dis.o ABSOLUTE
    ..\..\..\..\src\ble\profile\server\vendor_service.c 0x00000000   Number         0  vendor_service.o ABSOLUTE
    ..\..\..\..\src\ble\profile\server\voice_service.c 0x00000000   Number         0  voice_service.o ABSOLUTE
    ..\..\..\..\src\dfu\dfu_application.c    0x00000000   Number         0  dfu_application.o ABSOLUTE
    ..\..\..\..\src\dfu\dfu_main.c           0x00000000   Number         0  dfu_main.o ABSOLUTE
    ..\..\..\..\src\dfu\dfu_task.c           0x00000000   Number         0  dfu_task.o ABSOLUTE
    ..\..\..\..\src\mcu\peripheral\rtl876x_adc.c 0x00000000   Number         0  rtl876x_adc.o ABSOLUTE
    ..\..\..\..\src\mcu\peripheral\rtl876x_aon_wdg.c 0x00000000   Number         0  rtl876x_aon_wdg.o ABSOLUTE
    ..\..\..\..\src\mcu\peripheral\rtl876x_codec.c 0x00000000   Number         0  rtl876x_codec.o ABSOLUTE
    ..\..\..\..\src\mcu\peripheral\rtl876x_gdma.c 0x00000000   Number         0  rtl876x_gdma.o ABSOLUTE
    ..\..\..\..\src\mcu\peripheral\rtl876x_gpio.c 0x00000000   Number         0  rtl876x_gpio.o ABSOLUTE
    ..\..\..\..\src\mcu\peripheral\rtl876x_i2s.c 0x00000000   Number         0  rtl876x_i2s.o ABSOLUTE
    ..\..\..\..\src\mcu\peripheral\rtl876x_io_dlps.c 0x00000000   Number         0  rtl876x_io_dlps.o ABSOLUTE
    ..\..\..\..\src\mcu\peripheral\rtl876x_ir.c 0x00000000   Number         0  rtl876x_ir.o ABSOLUTE
    ..\..\..\..\src\mcu\peripheral\rtl876x_keyscan.c 0x00000000   Number         0  rtl876x_keyscan.o ABSOLUTE
    ..\..\..\..\src\mcu\peripheral\rtl876x_lpc.c 0x00000000   Number         0  rtl876x_lpc.o ABSOLUTE
    ..\..\..\..\src\mcu\peripheral\rtl876x_nvic.c 0x00000000   Number         0  rtl876x_nvic.o ABSOLUTE
    ..\..\..\..\src\mcu\peripheral\rtl876x_pinmux.c 0x00000000   Number         0  rtl876x_pinmux.o ABSOLUTE
    ..\..\..\..\src\mcu\peripheral\rtl876x_rcc.c 0x00000000   Number         0  rtl876x_rcc.o ABSOLUTE
    ..\..\..\..\src\mcu\peripheral\rtl876x_rtc.c 0x00000000   Number         0  rtl876x_rtc.o ABSOLUTE
    ..\..\..\..\src\mcu\peripheral\rtl876x_tim.c 0x00000000   Number         0  rtl876x_tim.o ABSOLUTE
    ..\..\..\..\src\mcu\peripheral\rtl876x_uart.c 0x00000000   Number         0  rtl876x_uart.o ABSOLUTE
    ..\..\..\..\src\mcu\rtl876x\overlay_mgr.c 0x00000000   Number         0  overlay_mgr.o ABSOLUTE
    ..\..\..\..\src\mcu\rtl876x\system_rtl876x.c 0x00000000   Number         0  system_rtl876x.o ABSOLUTE
    ..\..\..\..\src\platform\dfu_flash.c     0x00000000   Number         0  dfu_flash.o ABSOLUTE
    ..\\..\\..\\..\\src\\app\\google_rcu\\address_module\\rcu_link_mgr.c 0x00000000   Number         0  rcu_link_mgr.o ABSOLUTE
    ..\\..\\..\\..\\src\\app\\google_rcu\\app_task.c 0x00000000   Number         0  app_task.o ABSOLUTE
    ..\\..\\..\\..\\src\\app\\google_rcu\\bat_module\\battery_driver.c 0x00000000   Number         0  battery_driver.o ABSOLUTE
    ..\\..\\..\\..\\src\\app\\google_rcu\\buzzer_module\\buzzer_driver.c 0x00000000   Number         0  buzzer_driver.o ABSOLUTE
    ..\\..\\..\\..\\src\\app\\google_rcu\\buzzer_module\\fms_service_handle.c 0x00000000   Number         0  fms_service_handle.o ABSOLUTE
    ..\\..\\..\\..\\src\\app\\google_rcu\\dtm_module\\rcu_dtm_app.c 0x00000000   Number         0  rcu_dtm_app.o ABSOLUTE
    ..\\..\\..\\..\\src\\app\\google_rcu\\frm_vpk\\frm_vpk_api\\frm_vpk_hal_sflash.c 0x00000000   Number         0  frm_vpk_hal_sflash.o ABSOLUTE
    ..\\..\\..\\..\\src\\app\\google_rcu\\frm_vpk\\frm_vpk_api\\frm_vpk_log.c 0x00000000   Number         0  frm_vpk_log.o ABSOLUTE
    ..\\..\\..\\..\\src\\app\\google_rcu\\frm_vpk\\src\\app_custom.c 0x00000000   Number         0  app_custom.o ABSOLUTE
    ..\\..\\..\\..\\src\\app\\google_rcu\\frm_vpk\\src\\app_flash_write.c 0x00000000   Number         0  app_flash_write.o ABSOLUTE
    ..\\..\\..\\..\\src\\app\\google_rcu\\ir_module\\ir_protocol_nec.c 0x00000000   Number         0  ir_protocol_nec.o ABSOLUTE
    ..\\..\\..\\..\\src\\app\\google_rcu\\ir_module\\ir_send_driver.c 0x00000000   Number         0  ir_send_driver.o ABSOLUTE
    ..\\..\\..\\..\\src\\app\\google_rcu\\ir_module\\ir_send_handle.c 0x00000000   Number         0  ir_send_handle.o ABSOLUTE
    ..\\..\\..\\..\\src\\app\\google_rcu\\ir_module\\ir_service_handle.c 0x00000000   Number         0  ir_service_handle.o ABSOLUTE
    ..\\..\\..\\..\\src\\app\\google_rcu\\key_module\\key_handle.c 0x00000000   Number         0  key_handle.o ABSOLUTE
    ..\\..\\..\\..\\src\\app\\google_rcu\\key_module\\keyscan_driver.c 0x00000000   Number         0  keyscan_driver.o ABSOLUTE
    ..\\..\\..\\..\\src\\app\\google_rcu\\led_module\\led_driver.c 0x00000000   Number         0  led_driver.o ABSOLUTE
    ..\\..\\..\\..\\src\\app\\google_rcu\\led_module\\led_pwm_driver.c 0x00000000   Number         0  led_pwm_driver.o ABSOLUTE
    ..\\..\\..\\..\\src\\app\\google_rcu\\loop_queue.c 0x00000000   Number         0  loop_queue.o ABSOLUTE
    ..\\..\\..\\..\\src\\app\\google_rcu\\main.c 0x00000000   Number         0  main.o ABSOLUTE
    ..\\..\\..\\..\\src\\app\\google_rcu\\profile_module\\dfu_service.c 0x00000000   Number         0  dfu_service.o ABSOLUTE
    ..\\..\\..\\..\\src\\app\\google_rcu\\profile_module\\fms.c 0x00000000   Number         0  fms.o ABSOLUTE
    ..\\..\\..\\..\\src\\app\\google_rcu\\profile_module\\hids_rmc.c 0x00000000   Number         0  hids_rmc.o ABSOLUTE
    ..\\..\\..\\..\\src\\app\\google_rcu\\profile_module\\ir_service.c 0x00000000   Number         0  ir_service.o ABSOLUTE
    ..\\..\\..\\..\\src\\app\\google_rcu\\profile_module\\ota_service.c 0x00000000   Number         0  ota_service.o ABSOLUTE
    ..\\..\\..\\..\\src\\app\\google_rcu\\rcu_application.c 0x00000000   Number         0  rcu_application.o ABSOLUTE
    ..\\..\\..\\..\\src\\app\\google_rcu\\rcu_gap.c 0x00000000   Number         0  rcu_gap.o ABSOLUTE
    ..\\..\\..\\..\\src\\app\\google_rcu\\reset_watch_dog_timer.c 0x00000000   Number         0  reset_watch_dog_timer.o ABSOLUTE
    ..\\..\\..\\..\\src\\app\\google_rcu\\rtc_module\\rtc_driver.c 0x00000000   Number         0  rtc_driver.o ABSOLUTE
    ..\\..\\..\\..\\src\\app\\google_rcu\\swtimer.c 0x00000000   Number         0  swtimer.o ABSOLUTE
    ..\\..\\..\\..\\src\\app\\google_rcu\\test_module\\data_uart_test.c 0x00000000   Number         0  data_uart_test.o ABSOLUTE
    ..\\..\\..\\..\\src\\app\\google_rcu\\test_module\\mp_test.c 0x00000000   Number         0  mp_test.o ABSOLUTE
    ..\\..\\..\\..\\src\\app\\google_rcu\\test_module\\single_tone.c 0x00000000   Number         0  single_tone.o ABSOLUTE
    ..\\..\\..\\..\\src\\app\\google_rcu\\test_module\\uart_transport.c 0x00000000   Number         0  uart_transport.o ABSOLUTE
    ..\\..\\..\\..\\src\\app\\google_rcu\\voice_module\\voice.c 0x00000000   Number         0  voice.o ABSOLUTE
    ..\\..\\..\\..\\src\\app\\google_rcu\\voice_module\\voice_driver.c 0x00000000   Number         0  voice_driver.o ABSOLUTE
    ..\\..\\..\\..\\src\\ble\\privacy\\privacy_mgnt.c 0x00000000   Number         0  privacy_mgnt.o ABSOLUTE
    ..\\..\\..\\..\\src\\ble\\profile\\server\\atvv_service.c 0x00000000   Number         0  atvv_service.o ABSOLUTE
    ..\\..\\..\\..\\src\\ble\\profile\\server\\bas.c 0x00000000   Number         0  bas.o ABSOLUTE
    ..\\..\\..\\..\\src\\ble\\profile\\server\\dis.c 0x00000000   Number         0  dis.o ABSOLUTE
    ..\\..\\..\\..\\src\\ble\\profile\\server\\vendor_service.c 0x00000000   Number         0  vendor_service.o ABSOLUTE
    ..\\..\\..\\..\\src\\ble\\profile\\server\\voice_service.c 0x00000000   Number         0  voice_service.o ABSOLUTE
    ..\\..\\..\\..\\src\\dfu\\dfu_application.c 0x00000000   Number         0  dfu_application.o ABSOLUTE
    ..\\..\\..\\..\\src\\dfu\\dfu_main.c     0x00000000   Number         0  dfu_main.o ABSOLUTE
    ..\\..\\..\\..\\src\\dfu\\dfu_task.c     0x00000000   Number         0  dfu_task.o ABSOLUTE
    ..\\..\\..\\..\\src\\mcu\\peripheral\\rtl876x_adc.c 0x00000000   Number         0  rtl876x_adc.o ABSOLUTE
    ..\\..\\..\\..\\src\\mcu\\peripheral\\rtl876x_aon_wdg.c 0x00000000   Number         0  rtl876x_aon_wdg.o ABSOLUTE
    ..\\..\\..\\..\\src\\mcu\\peripheral\\rtl876x_codec.c 0x00000000   Number         0  rtl876x_codec.o ABSOLUTE
    ..\\..\\..\\..\\src\\mcu\\peripheral\\rtl876x_gdma.c 0x00000000   Number         0  rtl876x_gdma.o ABSOLUTE
    ..\\..\\..\\..\\src\\mcu\\peripheral\\rtl876x_gpio.c 0x00000000   Number         0  rtl876x_gpio.o ABSOLUTE
    ..\\..\\..\\..\\src\\mcu\\peripheral\\rtl876x_i2s.c 0x00000000   Number         0  rtl876x_i2s.o ABSOLUTE
    ..\\..\\..\\..\\src\\mcu\\peripheral\\rtl876x_io_dlps.c 0x00000000   Number         0  rtl876x_io_dlps.o ABSOLUTE
    ..\\..\\..\\..\\src\\mcu\\peripheral\\rtl876x_ir.c 0x00000000   Number         0  rtl876x_ir.o ABSOLUTE
    ..\\..\\..\\..\\src\\mcu\\peripheral\\rtl876x_keyscan.c 0x00000000   Number         0  rtl876x_keyscan.o ABSOLUTE
    ..\\..\\..\\..\\src\\mcu\\peripheral\\rtl876x_lpc.c 0x00000000   Number         0  rtl876x_lpc.o ABSOLUTE
    ..\\..\\..\\..\\src\\mcu\\peripheral\\rtl876x_nvic.c 0x00000000   Number         0  rtl876x_nvic.o ABSOLUTE
    ..\\..\\..\\..\\src\\mcu\\peripheral\\rtl876x_pinmux.c 0x00000000   Number         0  rtl876x_pinmux.o ABSOLUTE
    ..\\..\\..\\..\\src\\mcu\\peripheral\\rtl876x_rcc.c 0x00000000   Number         0  rtl876x_rcc.o ABSOLUTE
    ..\\..\\..\\..\\src\\mcu\\peripheral\\rtl876x_rtc.c 0x00000000   Number         0  rtl876x_rtc.o ABSOLUTE
    ..\\..\\..\\..\\src\\mcu\\peripheral\\rtl876x_tim.c 0x00000000   Number         0  rtl876x_tim.o ABSOLUTE
    ..\\..\\..\\..\\src\\mcu\\peripheral\\rtl876x_uart.c 0x00000000   Number         0  rtl876x_uart.o ABSOLUTE
    ..\\..\\..\\..\\src\\mcu\\rtl876x\\arm\\startup_rtl876x.s 0x00000000   Number         0  startup_rtl876x.o ABSOLUTE
    ..\\..\\..\\..\\src\\mcu\\rtl876x\\system_rtl876x.c 0x00000000   Number         0  system_rtl876x.o ABSOLUTE
    ..\\..\\..\\..\\src\\platform\\dfu_flash.c 0x00000000   Number         0  dfu_flash.o ABSOLUTE
    source\ima_adpcm_enc.c                   0x00000000   Number         0  ima_adpcm_enc.o ABSOLUTE
    VECTOR                                   0x00200000   Section      232  startup_rtl876x.o(VECTOR)
    .app.data_ram.text                       0x00207c00   Section        0  system_rtl876x.o(.app.data_ram.text)
    .app.data_ram.text                       0x00207d14   Section        0  rtl876x_io_dlps.o(.app.data_ram.text)
    TIM_DLPS_Enter                           0x00207d15   Thumb Code   138  rtl876x_io_dlps.o(.app.data_ram.text)
    GPIO_DLPS_Enter                          0x00207fb7   Thumb Code    74  rtl876x_io_dlps.o(.app.data_ram.text)
    GPIO_DLPS_Exit                           0x00208001   Thumb Code    80  rtl876x_io_dlps.o(.app.data_ram.text)
    KeyScan_DLPS_Exit                        0x00208051   Thumb Code    90  rtl876x_io_dlps.o(.app.data_ram.text)
    TIM_DLPS_Exit                            0x002080ab   Thumb Code   182  rtl876x_io_dlps.o(.app.data_ram.text)
    .app.data_ram.text                       0x00208164   Section        0  main.o(.app.data_ram.text)
    app_enter_dlps_config                    0x00208165 * Thumb Code    32  main.o(.app.data_ram.text)
    app_exit_dlps_config                     0x00208185 * Thumb Code    36  main.o(.app.data_ram.text)
    app_dlps_check_cb                        0x002081a9 * Thumb Code    42  main.o(.app.data_ram.text)
    .app.data_ram.text                       0x00208228   Section        0  rcu_application.o(.app.data_ram.text)
    .app.data_ram.text                       0x002082fc   Section        0  swtimer.o(.app.data_ram.text)
    back_key_pressed_when_HW_reset_timer_cb  0x002082fd * Thumb Code    20  swtimer.o(.app.data_ram.text)
    temp_off_latency_timer_cb                0x00208311 * Thumb Code    22  swtimer.o(.app.data_ram.text)
    adv_timer_callback                       0x00208327 * Thumb Code    26  swtimer.o(.app.data_ram.text)
    adv_change_data_timer_callback           0x00208341 * Thumb Code    20  swtimer.o(.app.data_ram.text)
    next_state_timeout_timer_callback        0x00208355 * Thumb Code    32  swtimer.o(.app.data_ram.text)
    update_conn_params_timer_cb              0x00208375 * Thumb Code    68  swtimer.o(.app.data_ram.text)
    aon_watch_dog_wake_up_dlps_callback      0x002083b9 * Thumb Code    16  swtimer.o(.app.data_ram.text)
    system_reset_timer_callback              0x002083c9 * Thumb Code    12  swtimer.o(.app.data_ram.text)
    .app.data_ram.text                       0x002083ec   Section        0  app_task.o(.app.data_ram.text)
    app_main_task                            0x002083ed * Thumb Code   134  app_task.o(.app.data_ram.text)
    .app.data_ram.text                       0x00208550   Section        0  reset_watch_dog_timer.o(.app.data_ram.text)
    .app.data_ram.text                       0x00208594   Section        0  loop_queue.o(.app.data_ram.text)
    .app.data_ram.text                       0x0020883c   Section        0  rtc_driver.o(.app.data_ram.text)
    .app.data_ram.text                       0x00208894   Section        0  keyscan_driver.o(.app.data_ram.text)
    keyscan_row_pad_config                   0x00208895   Thumb Code    44  keyscan_driver.o(.app.data_ram.text)
    keyscan_column_pad_config                0x002088c1   Thumb Code    44  keyscan_driver.o(.app.data_ram.text)
    keyscan_timer_callback                   0x00208b3d * Thumb Code    10  keyscan_driver.o(.app.data_ram.text)
    .app.data_ram.text                       0x00208b68   Section        0  key_handle.o(.app.data_ram.text)
    key_handle_comb_keys_timer_cb            0x00208b69 * Thumb Code    90  key_handle.o(.app.data_ram.text)
    notify_key_data_timer_cb                 0x00208bc3 * Thumb Code   138  key_handle.o(.app.data_ram.text)
    long_press_key_detect_timer_cb           0x00208c4d * Thumb Code    26  key_handle.o(.app.data_ram.text)
    .app.data_ram.text                       0x00208c7c   Section        0  voice_driver.o(.app.data_ram.text)
    .app.data_ram.text                       0x00208ce8   Section        0  voice.o(.app.data_ram.text)
    voice_handle_exception_timer_cb          0x00208ce9 * Thumb Code    54  voice.o(.app.data_ram.text)
    .app.data_ram.text                       0x00208d30   Section        0  ir_send_driver.o(.app.data_ram.text)
    ir_send_int_handler                      0x00208d31 * Thumb Code    96  ir_send_driver.o(.app.data_ram.text)
    ir_send_rtc_handler                      0x00208d91 * Thumb Code    50  ir_send_driver.o(.app.data_ram.text)
    .app.data_ram.text                       0x00208e28   Section        0  led_driver.o(.app.data_ram.text)
    led_ctrl_timer_cb                        0x00208e29 * Thumb Code   230  led_driver.o(.app.data_ram.text)
    .app.data_ram.text                       0x00208f1c   Section        0  fms_service_handle.o(.app.data_ram.text)
    fms_periodical_conn_callback             0x00208f1d * Thumb Code    40  fms_service_handle.o(.app.data_ram.text)
    .app.data_ram.text                       0x00208f4c   Section        0  battery_driver.o(.app.data_ram.text)
    bat_lpc_handler                          0x00208f4d * Thumb Code    70  battery_driver.o(.app.data_ram.text)
    .app.data_ram.text                       0x00209050   Section        0  frm_vpk_log.o(.app.data_ram.text)
    .text                                    0x0020908c   Section        0  rtl876x_io_dlps.o(.text)
    .data                                    0x002090a8   Section       46  dis.o(.data)
    dis_ieee_data_list_len                   0x002090a8   Data           1  dis.o(.data)
    dis_pnp_id                               0x002090a9   Data           7  dis.o(.data)
    dis_system_id                            0x002090b0   Data           8  dis.o(.data)
    dis_ieee_data_list                       0x002090b8   Data          30  dis.o(.data)
    .data                                    0x002090d6   Section        8  hids_rmc.o(.data)
    hids_protocol_mode                       0x002090d6   Data           1  hids_rmc.o(.data)
    hids_info                                0x002090da   Data           4  hids_rmc.o(.data)
    .data                                    0x002090e0   Section      168  dfu_service.o(.data)
    .data                                    0x00209188   Section        4  main.o(.data)
    .data                                    0x0020918c   Section       14  rcu_gap.o(.data)
    google_wake_adv_data_len                 0x0020918c   Data           1  rcu_gap.o(.data)
    google_wake_adv_data                     0x0020918d   Data          13  rcu_gap.o(.data)
    .data                                    0x0020919a   Section        2  privacy_mgnt.o(.data)
    .data                                    0x0020919c   Section      108  overlay_mgr.o(.data)
    overlay_sections                         0x0020919c   Data         108  overlay_mgr.o(.data)
    .data                                    0x00209208   Section        1  rcu_dtm_app.o(.data)
    phy                                      0x00209208   Data           1  rcu_dtm_app.o(.data)
    .data                                    0x00209209   Section        1  dfu_flash.o(.data)
    .data                                    0x0020920a   Section       14  keyscan_driver.o(.data)
    KeyScanRowPINs                           0x0020920a   Data           7  keyscan_driver.o(.data)
    KeyScanColumnPINs                        0x00209211   Data           7  keyscan_driver.o(.data)
    .data                                    0x00209218   Section       24  key_handle.o(.data)
    .data                                    0x00209230   Section       48  key_handle.o(.data)
    .data                                    0x00209260   Section        1  ir_send_handle.o(.data)
    ir_send_key_state                        0x00209260   Data           1  ir_send_handle.o(.data)
    .data                                    0x00209264   Section       20  ir_service_handle.o(.data)
    IR_Table_FTL_Addr_Info                   0x00209264   Data          20  ir_service_handle.o(.data)
    .data                                    0x00209278   Section        2  fms_service_handle.o(.data)
    Fms_Current_Mode                         0x00209278   Data           2  fms_service_handle.o(.data)
    .data                                    0x0020927c   Section        4  app_custom.o(.data)
    .data                                    0x00209280   Section       50  adc_lib.o(.data)
    .data                                    0x002092b4   Section      420  ima_adpcm_enc.o(.data)
    indexTable                               0x002092b4   Data          64  ima_adpcm_enc.o(.data)
    stepsizeTable                            0x002092f4   Data         356  ima_adpcm_enc.o(.data)
    .bss                                     0x00209458   Section       20  system_rtl876x.o(.bss)
    .bss                                     0x0020946c   Section      304  rtl876x_io_dlps.o(.bss)
    .bss                                     0x0020959c   Section        1  rtl876x_rtc.o(.bss)
    is_called                                0x0020959c   Data           1  rtl876x_rtc.o(.bss)
    .bss                                     0x0020959d   Section        1  rtl876x_lpc.o(.bss)
    is_called                                0x0020959d   Data           1  rtl876x_lpc.o(.bss)
    .bss                                     0x0020959e   Section        1  rtl876x_aon_wdg.o(.bss)
    is_called                                0x0020959e   Data           1  rtl876x_aon_wdg.o(.bss)
    .bss                                     0x002095a0   Section      132  dis.o(.bss)
    dis_manufacturer_name_len                0x002095a0   Data           1  dis.o(.bss)
    dis_model_number_len                     0x002095a1   Data           1  dis.o(.bss)
    dis_serial_number_len                    0x002095a2   Data           1  dis.o(.bss)
    dis_hardware_rev_len                     0x002095a3   Data           1  dis.o(.bss)
    dis_firmware_rev_len                     0x002095a4   Data           1  dis.o(.bss)
    dis_software_rev_len                     0x002095a5   Data           1  dis.o(.bss)
    pfn_dis_cb                               0x002095a8   Data           4  dis.o(.bss)
    dis_manufacturer_name                    0x002095ac   Data          20  dis.o(.bss)
    dis_model_number                         0x002095c0   Data          20  dis.o(.bss)
    dis_serial_number                        0x002095d4   Data          20  dis.o(.bss)
    dis_hardware_rev                         0x002095e8   Data          20  dis.o(.bss)
    dis_firmware_rev                         0x002095fc   Data          20  dis.o(.bss)
    dis_software_rev                         0x00209610   Data          20  dis.o(.bss)
    .bss                                     0x00209624   Section        8  bas.o(.bss)
    battery_level                            0x00209624   Data           1  bas.o(.bss)
    bas_read_battery_level_pending           0x00209625   Data           1  bas.o(.bss)
    pfn_bas_cb                               0x00209628   Data           4  bas.o(.bss)
    .bss                                     0x0020962c   Section       12  hids_rmc.o(.bss)
    hids_suspand_mode                        0x0020962c   Data           1  hids_rmc.o(.bss)
    RmcDataLen                               0x0020962e   Data           2  hids_rmc.o(.bss)
    pfn_hids_cb                              0x00209630   Data           4  hids_rmc.o(.bss)
    p_report_data                            0x00209634   Data           4  hids_rmc.o(.bss)
    .bss                                     0x00209638   Section       16  vendor_service.o(.bss)
    .bss                                     0x00209648   Section        4  vendor_service.o(.bss)
    pfn_vendor_svc_cb                        0x00209648   Data           4  vendor_service.o(.bss)
    .bss                                     0x0020964c   Section       74  atvv_service.o(.bss)
    pfn_atvv_cb                              0x0020964c   Data           4  atvv_service.o(.bss)
    .bss                                     0x00209698   Section        4  ir_service.o(.bss)
    pfn_ir_svc_cb                            0x00209698   Data           4  ir_service.o(.bss)
    .bss                                     0x0020969c   Section     2220  dfu_service.o(.bss)
    buffer_check_en                          0x0020969d   Data           1  dfu_service.o(.bss)
    dfu_service_id                           0x0020969e   Data           1  dfu_service.o(.bss)
    dfu_resend_offset                        0x002096a4   Data           4  dfu_service.o(.bss)
    .bss                                     0x00209f48   Section       88  ota_service.o(.bss)
    image_version                            0x00209f68   Data          44  ota_service.o(.bss)
    DeviceInfo                               0x00209f94   Data          12  ota_service.o(.bss)
    .bss                                     0x00209fa0   Section        8  fms.o(.bss)
    Fms_Ctl_mode                             0x00209fa0   Data           2  fms.o(.bss)
    pfn_fms_cb                               0x00209fa4   Data           4  fms.o(.bss)
    .bss                                     0x00209fa8   Section      180  rcu_application.o(.bss)
    .bss                                     0x0020a05c   Section       96  rcu_gap.o(.bss)
    app_scan_rsp_data_len                    0x0020a05c   Data           1  rcu_gap.o(.bss)
    app_pairing_adv_data_len                 0x0020a05d   Data           1  rcu_gap.o(.bss)
    custom_wakeup_adv_data_len               0x0020a05e   Data           1  rcu_gap.o(.bss)
    app_scan_rsp_data                        0x0020a05f   Data          31  rcu_gap.o(.bss)
    app_pairing_adv_data                     0x0020a07e   Data          31  rcu_gap.o(.bss)
    custom_wakeup_adv_data                   0x0020a09d   Data          31  rcu_gap.o(.bss)
    .bss                                     0x0020a0bc   Section       32  swtimer.o(.bss)
    .bss                                     0x0020a0dc   Section       16  app_task.o(.bss)
    .bss                                     0x0020a0ec   Section       16  privacy_mgnt.o(.bss)
    privacy_app_cb                           0x0020a0f4   Data           4  privacy_mgnt.o(.bss)
    .bss                                     0x0020a0fc   Section        8  overlay_mgr.o(.bss)
    .bss                                     0x0020a104   Section       10  rcu_dtm_app.o(.bss)
    up_2_bits                                0x0020a104   Data           1  rcu_dtm_app.o(.bss)
    mod_idx                                  0x0020a105   Data           1  rcu_dtm_app.o(.bss)
    lcl_feats                                0x0020a106   Data           8  rcu_dtm_app.o(.bss)
    .bss                                     0x0020a110   Section        8  rtc_driver.o(.bss)
    rtc_ovf_cnt                              0x0020a110   Data           4  rtc_driver.o(.bss)
    rtc_driver_comp_0_cb                     0x0020a114   Data           4  rtc_driver.o(.bss)
    .bss                                     0x0020a118   Section       12  dfu_flash.o(.bss)
    img_total_len                            0x0020a118   Data           4  dfu_flash.o(.bss)
    total_block_cnt                          0x0020a11c   Data           4  dfu_flash.o(.bss)
    block_cnt                                0x0020a120   Data           4  dfu_flash.o(.bss)
    .bss                                     0x0020a124   Section       48  keyscan_driver.o(.bss)
    keyscan_timer                            0x0020a124   Data           4  keyscan_driver.o(.bss)
    .bss                                     0x0020a154   Section      552  key_handle.o(.bss)
    current_cache_fifo_items_cnt             0x0020a154   Data           1  key_handle.o(.bss)
    cache_fifo_output_cnt                    0x0020a155   Data           1  key_handle.o(.bss)
    Key_Press_Cache_FIFO                     0x0020a164   Data          22  key_handle.o(.bss)
    .bss                                     0x0020a37c   Section     1128  voice_driver.o(.bss)
    voice_driver_gdma_link_list              0x0020a37c   Data          40  voice_driver.o(.bss)
    .bss                                     0x0020a7e4   Section       16  voice.o(.bss)
    voice_exception_timer                    0x0020a7e4   Data           4  voice.o(.bss)
    p_voice_queue                            0x0020a7e8   Data           4  voice.o(.bss)
    .bss                                     0x0020a7f4   Section        8  ir_send_driver.o(.bss)
    ir_send_struct                           0x0020a7f4   Data           8  ir_send_driver.o(.bss)
    .bss                                     0x0020a7fc   Section     1628  ir_send_handle.o(.bss)
    ir_send_parameters                       0x0020a7fc   Data        1628  ir_send_handle.o(.bss)
    .bss                                     0x0020ae58   Section     2568  ir_service_handle.o(.bss)
    ir_programing_timer                      0x0020ae58   Data           4  ir_service_handle.o(.bss)
    ir_table                                 0x0020ae5c   Data        2540  ir_service_handle.o(.bss)
    .bss                                     0x0020b860   Section       40  led_driver.o(.bss)
    led_global_tick_cnt                      0x0020b860   Data           4  led_driver.o(.bss)
    led_ctrl_timer                           0x0020b864   Data           4  led_driver.o(.bss)
    led_ctrl_data                            0x0020b868   Data          32  led_driver.o(.bss)
    .bss                                     0x0020b888   Section        2  led_pwm_driver.o(.bss)
    led_pwm_init_states                      0x0020b888   Data           1  led_pwm_driver.o(.bss)
    led_on_off_states                        0x0020b889   Data           1  led_pwm_driver.o(.bss)
    .bss                                     0x0020b88c   Section       12  buzzer_driver.o(.bss)
    .bss                                     0x0020b898   Section        8  fms_service_handle.o(.bss)
    Fms_Handle_Notify_Flag                   0x0020b898   Data           1  fms_service_handle.o(.bss)
    Fms_Periodical_Conn_Timer                0x0020b89c   Data           4  fms_service_handle.o(.bss)
    .bss                                     0x0020b8a0   Section        6  battery_driver.o(.bss)
    cur_bat_info                             0x0020b8a0   Data           6  battery_driver.o(.bss)
    .bss                                     0x0020b8a8   Section        8  gap_lib_system_call.o(.bss)
    .bss                                     0x0020b8b0   Section       84  adc_lib.o(.bss)
    .bss                                     0x0020b904   Section        6  ima_adpcm_enc.o(.bss)
    .bss                                     0x0020b90c   Section      228  rand.o(.bss)
    .bss                                     0x0020b9f0   Section       20  rt_locale.o(.bss)
    __rt_locale_data                         0x0020b9f0   Data          20  rt_locale.o(.bss)
    .app.overlay_a                           0x0020ba04   Section        0  system_rtl876x.o(.app.overlay_a)
    .app.flash.header                        0x00832000   Section     1024  system_rtl876x.o(.app.flash.header)
    __tagsym$$used                           0x00832000   Number         0  system_rtl876x.o(.app.flash.header)
    __tagsym$$used                           0x008321e0   Number         0  system_rtl876x.o(.app.flash.header)
    RESET                                    0x00832400   Section        8  startup_rtl876x.o(RESET)
    !!!main                                  0x00832408   Section        8  __main.o(!!!main)
    .ARM.Collect$$_printf_percent$$00000000  0x00832410   Section        2  _printf_percent.o(.ARM.Collect$$_printf_percent$$00000000)
    .ARM.Collect$$_printf_percent$$00000001  0x00832412   Section       10  _printf_n.o(.ARM.Collect$$_printf_percent$$00000001)
    .ARM.Collect$$_printf_percent$$00000002  0x0083241c   Section       10  _printf_p.o(.ARM.Collect$$_printf_percent$$00000002)
    .ARM.Collect$$_printf_percent$$00000003  0x00832426   Section       10  _printf_f.o(.ARM.Collect$$_printf_percent$$00000003)
    .ARM.Collect$$_printf_percent$$00000004  0x00832430   Section       10  _printf_e.o(.ARM.Collect$$_printf_percent$$00000004)
    .ARM.Collect$$_printf_percent$$00000005  0x0083243a   Section       10  _printf_g.o(.ARM.Collect$$_printf_percent$$00000005)
    .ARM.Collect$$_printf_percent$$00000006  0x00832444   Section       10  _printf_a.o(.ARM.Collect$$_printf_percent$$00000006)
    .ARM.Collect$$_printf_percent$$00000007  0x0083244e   Section       10  _printf_ll.o(.ARM.Collect$$_printf_percent$$00000007)
    .ARM.Collect$$_printf_percent$$00000008  0x00832458   Section       10  _printf_i.o(.ARM.Collect$$_printf_percent$$00000008)
    .ARM.Collect$$_printf_percent$$00000009  0x00832462   Section       10  _printf_d.o(.ARM.Collect$$_printf_percent$$00000009)
    .ARM.Collect$$_printf_percent$$0000000A  0x0083246c   Section       10  _printf_u.o(.ARM.Collect$$_printf_percent$$0000000A)
    .ARM.Collect$$_printf_percent$$0000000B  0x00832476   Section       10  _printf_o.o(.ARM.Collect$$_printf_percent$$0000000B)
    .ARM.Collect$$_printf_percent$$0000000C  0x00832480   Section       10  _printf_x.o(.ARM.Collect$$_printf_percent$$0000000C)
    .ARM.Collect$$_printf_percent$$0000000D  0x0083248a   Section       10  _printf_lli.o(.ARM.Collect$$_printf_percent$$0000000D)
    .ARM.Collect$$_printf_percent$$0000000E  0x00832494   Section       10  _printf_lld.o(.ARM.Collect$$_printf_percent$$0000000E)
    .ARM.Collect$$_printf_percent$$0000000F  0x0083249e   Section       10  _printf_llu.o(.ARM.Collect$$_printf_percent$$0000000F)
    .ARM.Collect$$_printf_percent$$00000010  0x008324a8   Section       10  _printf_llo.o(.ARM.Collect$$_printf_percent$$00000010)
    .ARM.Collect$$_printf_percent$$00000011  0x008324b2   Section       10  _printf_llx.o(.ARM.Collect$$_printf_percent$$00000011)
    .ARM.Collect$$_printf_percent$$00000012  0x008324bc   Section       10  _printf_l.o(.ARM.Collect$$_printf_percent$$00000012)
    .ARM.Collect$$_printf_percent$$00000013  0x008324c6   Section       10  _printf_c.o(.ARM.Collect$$_printf_percent$$00000013)
    .ARM.Collect$$_printf_percent$$00000014  0x008324d0   Section       10  _printf_s.o(.ARM.Collect$$_printf_percent$$00000014)
    .ARM.Collect$$_printf_percent$$00000015  0x008324da   Section       10  _printf_lc.o(.ARM.Collect$$_printf_percent$$00000015)
    .ARM.Collect$$_printf_percent$$00000016  0x008324e4   Section       10  _printf_ls.o(.ARM.Collect$$_printf_percent$$00000016)
    .ARM.Collect$$_printf_percent$$00000017  0x008324ee   Section        4  _printf_percent_end.o(.ARM.Collect$$_printf_percent$$00000017)
    .ARM.Collect$$libinit$$00000000          0x008324f2   Section        2  libinit.o(.ARM.Collect$$libinit$$00000000)
    .ARM.Collect$$libinit$$00000002          0x008324f4   Section        0  libinit2.o(.ARM.Collect$$libinit$$00000002)
    .ARM.Collect$$libinit$$00000004          0x008324f4   Section        0  libinit2.o(.ARM.Collect$$libinit$$00000004)
    .ARM.Collect$$libinit$$0000000A          0x008324f4   Section        0  libinit2.o(.ARM.Collect$$libinit$$0000000A)
    .ARM.Collect$$libinit$$0000000C          0x008324f4   Section        0  libinit2.o(.ARM.Collect$$libinit$$0000000C)
    .ARM.Collect$$libinit$$0000000D          0x008324f4   Section        4  libinit2.o(.ARM.Collect$$libinit$$0000000D)
    .ARM.Collect$$libinit$$0000000E          0x008324f8   Section        0  libinit2.o(.ARM.Collect$$libinit$$0000000E)
    .ARM.Collect$$libinit$$0000000F          0x008324f8   Section        6  libinit2.o(.ARM.Collect$$libinit$$0000000F)
    .ARM.Collect$$libinit$$00000011          0x008324fe   Section        0  libinit2.o(.ARM.Collect$$libinit$$00000011)
    .ARM.Collect$$libinit$$00000012          0x008324fe   Section       12  libinit2.o(.ARM.Collect$$libinit$$00000012)
    .ARM.Collect$$libinit$$00000013          0x0083250a   Section        0  libinit2.o(.ARM.Collect$$libinit$$00000013)
    .ARM.Collect$$libinit$$00000015          0x0083250a   Section        0  libinit2.o(.ARM.Collect$$libinit$$00000015)
    .ARM.Collect$$libinit$$00000016          0x0083250a   Section       10  libinit2.o(.ARM.Collect$$libinit$$00000016)
    .ARM.Collect$$libinit$$00000017          0x00832514   Section        0  libinit2.o(.ARM.Collect$$libinit$$00000017)
    .ARM.Collect$$libinit$$00000019          0x00832514   Section        0  libinit2.o(.ARM.Collect$$libinit$$00000019)
    .ARM.Collect$$libinit$$0000001B          0x00832514   Section        0  libinit2.o(.ARM.Collect$$libinit$$0000001B)
    .ARM.Collect$$libinit$$0000001D          0x00832514   Section        0  libinit2.o(.ARM.Collect$$libinit$$0000001D)
    .ARM.Collect$$libinit$$0000001F          0x00832514   Section        0  libinit2.o(.ARM.Collect$$libinit$$0000001F)
    .ARM.Collect$$libinit$$00000021          0x00832514   Section        0  libinit2.o(.ARM.Collect$$libinit$$00000021)
    .ARM.Collect$$libinit$$00000023          0x00832514   Section        0  libinit2.o(.ARM.Collect$$libinit$$00000023)
    .ARM.Collect$$libinit$$00000025          0x00832514   Section        0  libinit2.o(.ARM.Collect$$libinit$$00000025)
    .ARM.Collect$$libinit$$0000002C          0x00832514   Section        0  libinit2.o(.ARM.Collect$$libinit$$0000002C)
    .ARM.Collect$$libinit$$0000002E          0x00832514   Section        0  libinit2.o(.ARM.Collect$$libinit$$0000002E)
    .ARM.Collect$$libinit$$00000030          0x00832514   Section        0  libinit2.o(.ARM.Collect$$libinit$$00000030)
    .ARM.Collect$$libinit$$00000032          0x00832514   Section        0  libinit2.o(.ARM.Collect$$libinit$$00000032)
    .ARM.Collect$$libinit$$00000033          0x00832514   Section        2  libinit2.o(.ARM.Collect$$libinit$$00000033)
    .ARM.Collect$$rtentry$$00000000          0x00832516   Section        0  __rtentry.o(.ARM.Collect$$rtentry$$00000000)
    .ARM.Collect$$rtentry$$00000002          0x00832516   Section        0  __rtentry2.o(.ARM.Collect$$rtentry$$00000002)
    .ARM.Collect$$rtentry$$00000005          0x00832516   Section        4  __rtentry5.o(.ARM.Collect$$rtentry$$00000005)
    .ARM.Collect$$rtentry$$00000009          0x0083251a   Section        0  __rtentry2.o(.ARM.Collect$$rtentry$$00000009)
    .ARM.Collect$$rtentry$$0000000A          0x0083251a   Section        4  __rtentry2.o(.ARM.Collect$$rtentry$$0000000A)
    .ARM.Collect$$rtentry$$0000000C          0x0083251e   Section        0  __rtentry2.o(.ARM.Collect$$rtentry$$0000000C)
    .ARM.Collect$$rtentry$$0000000D          0x0083251e   Section        8  __rtentry2.o(.ARM.Collect$$rtentry$$0000000D)
    .ARM.Collect$$rtentry$$00002716          0x00832528   Section        4  __rtentry5.o(.ARM.Collect$$rtentry$$00002716)
    __lit__00000000                          0x00832528   Data           4  __rtentry5.o(.ARM.Collect$$rtentry$$00002716)
    .app.flash.text                          0x0083252c   Section        0  system_rtl876x.o(.app.flash.text)
    .text                                    0x00832904   Section       84  startup_rtl876x.o(.text)
    DEFAULT_HANDLER_TXT                      0x00832914   Data           0  startup_rtl876x.o(.text)
    .text                                    0x00832958   Section        0  system_rtl876x.o(.text)
    .text                                    0x00832b34   Section        0  rtl876x_gpio.o(.text)
    .text                                    0x00832cc8   Section        0  rtl876x_ir.o(.text)
    .text                                    0x00832fc0   Section        0  rtl876x_keyscan.o(.text)
    .text                                    0x00833160   Section        0  rtl876x_rtc.o(.text)
    .text                                    0x008333bc   Section        0  rtl876x_codec.o(.text)
    .text                                    0x00833700   Section        0  rtl876x_i2s.o(.text)
    .text                                    0x00833830   Section        0  rtl876x_pinmux.o(.text)
    .text                                    0x00833b98   Section        0  rtl876x_nvic.o(.text)
    .text                                    0x00833c60   Section        0  rtl876x_rcc.o(.text)
    .text                                    0x00833f70   Section        0  rtl876x_tim.o(.text)
    .text                                    0x0083410c   Section        0  rtl876x_gdma.o(.text)
    GDMA_GetSuspendChannelStatus             0x0083441b   Thumb Code    14  rtl876x_gdma.o(.text)
    .text                                    0x00834440   Section        0  rtl876x_uart.o(.text)
    .text                                    0x00834694   Section        0  rtl876x_adc.o(.text)
    .text                                    0x008349a0   Section        0  rtl876x_lpc.o(.text)
    .text                                    0x00834bec   Section        0  rtl876x_aon_wdg.o(.text)
    AON_WDG_WriteReg                         0x00834bed   Thumb Code    38  rtl876x_aon_wdg.o(.text)
    .text                                    0x00834e14   Section        0  dis.o(.text)
    .text                                    0x00835080   Section        0  bas.o(.text)
    .text                                    0x008351ec   Section        0  hids_rmc.o(.text)
    .text                                    0x00835454   Section        0  vendor_service.o(.text)
    .text                                    0x00835564   Section        0  atvv_service.o(.text)
    .text                                    0x00835710   Section        0  ir_service.o(.text)
    .text                                    0x00835814   Section        0  dfu_service.o(.text)
    buf_swap                                 0x0083654f   Thumb Code    32  dfu_service.o(.text)
    .text                                    0x00836584   Section        0  ota_service.o(.text)
    get_ota_active_bank_image_info           0x0083661d   Thumb Code   108  ota_service.o(.text)
    .text                                    0x00836a04   Section        0  fms.o(.text)
    .text                                    0x00836b30   Section        0  main.o(.text)
    global_data_init                         0x00836b3d   Thumb Code   348  main.o(.text)
    app_normal_power_on_seq                  0x00836dc9   Thumb Code   108  main.o(.text)
    app_le_profile_init                      0x00836e35   Thumb Code   100  main.o(.text)
    .text                                    0x00836ee8   Section        0  rcu_application.o(.text)
    app_stop_adv_reason_handler              0x00836ee9   Thumb Code   256  rcu_application.o(.text)
    app_disconn_reason_handler               0x00836fe9   Thumb Code   150  rcu_application.o(.text)
    app_dis_srv_cb                           0x00837141   Thumb Code   200  rcu_application.o(.text)
    app_dfu_srv_cb                           0x00837209   Thumb Code   368  rcu_application.o(.text)
    periph_handle_dev_state_evt              0x00837379   Thumb Code   350  rcu_application.o(.text)
    periph_handle_conn_state_evt             0x008374d7   Thumb Code   314  rcu_application.o(.text)
    periph_handle_authen_state_evt           0x00837611   Thumb Code   240  rcu_application.o(.text)
    periph_conn_param_update_evt             0x00837701   Thumb Code   248  rcu_application.o(.text)
    periph_handle_gap_msg                    0x008377f9   Thumb Code   322  rcu_application.o(.text)
    app_general_srv_cb                       0x00837c39   Thumb Code   118  rcu_application.o(.text)
    app_hid_srv_cb                           0x00837caf   Thumb Code   136  rcu_application.o(.text)
    app_vendor_srv_cb                        0x00837d37   Thumb Code   158  rcu_application.o(.text)
    .text                                    0x00837df8   Section        0  rcu_gap.o(.text)
    .text                                    0x008388f4   Section        0  swtimer.o(.text)
    .text                                    0x00838b4c   Section        0  app_task.o(.text)
    .text                                    0x00838b9c   Section        0  reset_watch_dog_timer.o(.text)
    .text                                    0x00838bfc   Section        0  privacy_mgnt.o(.text)
    .text                                    0x00839308   Section        0  overlay_mgr.o(.text)
    .text                                    0x00839384   Section        0  loop_queue.o(.text)
    .text                                    0x00839418   Section        0  rcu_dtm_app.o(.text)
    .text                                    0x0083984c   Section        0  rtc_driver.o(.text)
    .text                                    0x008399a8   Section        0  dfu_flash.o(.text)
    dfu_write                                0x008399c5   Thumb Code   180  dfu_flash.o(.text)
    flash_erase_sector                       0x00839f3f   Thumb Code    32  dfu_flash.o(.text)
    flash_erase_block                        0x00839f5f   Thumb Code    34  dfu_flash.o(.text)
    dfu_flash_check_blank                    0x00839f81   Thumb Code   136  dfu_flash.o(.text)
    check_dfu_update_image_length            0x0083a009   Thumb Code   110  dfu_flash.o(.text)
    .text                                    0x0083a0c4   Section        0  keyscan_driver.o(.text)
    keyscan_disable_wakeup_config            0x0083a143   Thumb Code    28  keyscan_driver.o(.text)
    .text                                    0x0083a188   Section        0  key_handle.o(.text)
    key_handle_prepare_hid_usage_buffer      0x0083a1ad   Thumb Code   140  key_handle.o(.text)
    key_handle_notify_hid_usage_buffer       0x0083a239   Thumb Code   208  key_handle.o(.text)
    key_handle_inqueue_key_pressed_cache_fifo 0x0083a331   Thumb Code    86  key_handle.o(.text)
    key_handle_process_factory_reset_event   0x0083a4af   Thumb Code    74  key_handle.o(.text)
    key_handle_one_key_scenario              0x0083a4f9   Thumb Code   498  key_handle.o(.text)
    key_handle_detect_special_keys           0x0083a7d5   Thumb Code   306  key_handle.o(.text)
    key_handle_process_repairing_event       0x0083ac73   Thumb Code    90  key_handle.o(.text)
    key_handle_check_navy_key                0x0083accd   Thumb Code    54  key_handle.o(.text)
    .text                                    0x0083ad54   Section        0  voice_driver.o(.text)
    voice_driver_init_rx_gdma                0x0083ad55   Thumb Code   238  voice_driver.o(.text)
    voice_driver_init_i2s                    0x0083af2d   Thumb Code   112  voice_driver.o(.text)
    voice_driver_init_codec                  0x0083af9d   Thumb Code   102  voice_driver.o(.text)
    .text                                    0x0083b030   Section        0  voice.o(.text)
    voice_handle_notify_voice_data           0x0083b031   Thumb Code   316  voice.o(.text)
    voice_handle_gdma_event                  0x0083b253   Thumb Code   182  voice.o(.text)
    voice_handle_atv_audio_sync              0x0083ba75   Thumb Code    98  voice.o(.text)
    voice_handle_encode_raw_data             0x0083bad7   Thumb Code    74  voice.o(.text)
    .text                                    0x0083bb54   Section        0  ir_send_driver.o(.text)
    ir_driver_tx_gdma_init                   0x0083bb55   Thumb Code   104  ir_send_driver.o(.text)
    ir_send_driver_init                      0x0083be09   Thumb Code   108  ir_send_driver.o(.text)
    .text                                    0x0083beb0   Section        0  ir_send_handle.o(.text)
    ir_send_command_encode                   0x0083c2bf   Thumb Code    62  ir_send_handle.o(.text)
    .text                                    0x0083c2fc   Section        0  ir_protocol_nec.o(.text)
    ir_protocol_nec_command_set_tx_buf       0x0083c2fd   Thumb Code   200  ir_protocol_nec.o(.text)
    hl_time2_tx_buf_count                    0x0083c46b   Thumb Code    32  ir_protocol_nec.o(.text)
    .text                                    0x0083c4a4   Section        0  ir_service_handle.o(.text)
    ir_service_handle_activate_ir_table      0x0083c4c5   Thumb Code    56  ir_service_handle.o(.text)
    ir_service_handle_write_prog_control_char 0x0083c59d   Thumb Code   174  ir_service_handle.o(.text)
    ir_service_handle_back_up_ftl_table      0x0083c66f   Thumb Code   154  ir_service_handle.o(.text)
    ir_service_handle_restore_ir_table_from_ftl 0x0083c709   Thumb Code   234  ir_service_handle.o(.text)
    ir_service_handle_write_char_cb          0x0083ca79   Thumb Code   142  ir_service_handle.o(.text)
    ir_service_handle_write_suppress_char    0x0083cb07   Thumb Code    86  ir_service_handle.o(.text)
    ir_service_handle_write_code_char        0x0083cb5d   Thumb Code    96  ir_service_handle.o(.text)
    ir_service_handle_ir_table_add_item      0x0083cbbd   Thumb Code   124  ir_service_handle.o(.text)
    .text                                    0x0083cc64   Section        0  led_driver.o(.text)
    .text                                    0x0083cd78   Section        0  led_pwm_driver.o(.text)
    led_module_update_pwm_states             0x0083cd79   Thumb Code    26  led_pwm_driver.o(.text)
    led_module_update_on_off_states          0x0083cd93   Thumb Code    26  led_pwm_driver.o(.text)
    .text                                    0x0083ced8   Section        0  buzzer_driver.o(.text)
    buzzer_init_driver                       0x0083cfc3   Thumb Code   128  buzzer_driver.o(.text)
    .text                                    0x0083d060   Section        0  fms_service_handle.o(.text)
    fms_handle_write_char_cb                 0x0083d1d5   Thumb Code    92  fms_service_handle.o(.text)
    fms_handle_write_data_char               0x0083d231   Thumb Code   134  fms_service_handle.o(.text)
    .text                                    0x0083d304   Section        0  battery_driver.o(.text)
    bat_calibrate_voltage                    0x0083d305   Thumb Code   122  battery_driver.o(.text)
    bat_driver_lpc_init                      0x0083d37f   Thumb Code   106  battery_driver.o(.text)
    bat_calculate_bat_level                  0x0083d675   Thumb Code   224  battery_driver.o(.text)
    bat_handle_key_pressed_event             0x0083d755   Thumb Code    72  battery_driver.o(.text)
    .text                                    0x0083d7a8   Section        0  app_custom.o(.text)
    .text                                    0x0083df14   Section        0  frm_vpk_hal_sflash.o(.text)
    .text                                    0x0083dfc0   Section        0  gap_lib_system_call.o(.text)
    .text                                    0x0083f08c   Section        0  adc_lib.o(.text)
    ADC_GetKValue                            0x0083f08d   Thumb Code    66  adc_lib.o(.text)
    ADC_GetKVoltage                          0x0083f0cf   Thumb Code    82  adc_lib.o(.text)
    .text                                    0x0083f398   Section        0  llmul.o(.text)
    .text                                    0x0083f3c8   Section        0  lludiv.o(.text)
    .text                                    0x0083f4cc   Section        0  vsprintf.o(.text)
    .text                                    0x0083f4f0   Section        0  rand.o(.text)
    .text                                    0x0083f52c   Section      346  aeabi_sdiv.o(.text)
    .text                                    0x0083f688   Section        0  d2f.o(.text)
    .text                                    0x0083f704   Section        0  daddsub.o(.text)
    _dadd1                                   0x0083f705   Thumb Code   290  daddsub.o(.text)
    _dsub1                                   0x0083f827   Thumb Code   470  daddsub.o(.text)
    .text                                    0x0083fa5c   Section        0  ddiv.o(.text)
    .text                                    0x0083fea4   Section        0  dfixui.o(.text)
    .text                                    0x0083feec   Section        0  dflti.o(.text)
    .text                                    0x0083ff44   Section        0  dmul.o(.text)
    .text                                    0x0084018c   Section        0  f2d.o(.text)
    .text                                    0x008401e0   Section        0  fdiv.o(.text)
    .text                                    0x00840340   Section        0  ffixui.o(.text)
    .text                                    0x00840370   Section        0  fflti.o(.text)
    .text                                    0x008403ce   Section        0  _printf_pad.o(.text)
    .text                                    0x0084041c   Section        0  _printf_truncate.o(.text)
    .text                                    0x00840440   Section        0  _printf_str.o(.text)
    .text                                    0x00840494   Section        0  _printf_dec.o(.text)
    .text                                    0x00840500   Section        0  _printf_charcount.o(.text)
    .text                                    0x00840528   Section        0  _printf_char_common.o(.text)
    _printf_input_char                       0x00840529   Thumb Code    10  _printf_char_common.o(.text)
    .text                                    0x00840558   Section        0  _sputc.o(.text)
    .text                                    0x00840564   Section        0  _printf_wctomb.o(.text)
    .text                                    0x00840620   Section        0  _printf_longlong_dec.o(.text)
    .text                                    0x00840690   Section        0  _printf_oct_int_ll.o(.text)
    _printf_longlong_oct_internal            0x00840691   Thumb Code     0  _printf_oct_int_ll.o(.text)
    .text                                    0x00840700   Section        0  _printf_hex_int_ll_ptr.o(.text)
    _printf_hex_common                       0x00840701   Thumb Code     0  _printf_hex_int_ll_ptr.o(.text)
    .text                                    0x00840798   Section        0  __printf_flags_ss_wp.o(.text)
    .text                                    0x00840920   Section        0  lludiv10.o(.text)
    .text                                    0x0084099a   Section        0  _printf_intcommon.o(.text)
    .text                                    0x00840a4c   Section        0  _printf_fp_dec.o(.text)
    _fp_digits                               0x00840a4f   Thumb Code   412  _printf_fp_dec.o(.text)
    .text                                    0x00840e64   Section        0  _printf_fp_hex.o(.text)
    .text                                    0x0084113c   Section        0  _printf_char.o(.text)
    .text                                    0x0084116a   Section        0  _printf_wchar.o(.text)
    .text                                    0x00841198   Section        0  _wcrtomb.o(.text)
    .text                                    0x008411d8   Section        0  rtudiv10.o(.text)
    .text                                    0x00841200   Section       16  rt_ctype_table.o(.text)
    .text                                    0x00841210   Section        8  rt_locale.o(.text)
    .text                                    0x00841218   Section        0  _printf_fp_infnan.o(.text)
    .text                                    0x008412a0   Section        0  bigflt0.o(.text)
    .text                                    0x00841378   Section        0  btod.o(.text)
    btod_internal_mul                        0x008413b9   Thumb Code   492  btod.o(.text)
    btod_internal_div                        0x008415a5   Thumb Code   520  btod.o(.text)
    .text                                    0x008418f8   Section        0  strcmp.o(.text)
    i.__ARM_common_ll_muluu                  0x00841980   Section        0  btod.o(i.__ARM_common_ll_muluu)
    i.__ARM_common_switch8                   0x008419b0   Section        0  dis.o(i.__ARM_common_switch8)
    i.__ARM_fpclassify                       0x008419cc   Section        0  fpclassify.o(i.__ARM_fpclassify)
    i._is_digit                              0x008419f8   Section        0  __printf_wp.o(i._is_digit)
    i.ima_adpcm_encode                       0x00841a08   Section        0  ima_adpcm_enc.o(i.ima_adpcm_encode)
    locale$$code                             0x00841b40   Section       44  lc_numeric_c.o(locale$$code)
    locale$$code                             0x00841b6c   Section       44  lc_ctype_c.o(locale$$code)
    x$fpl$fadd                               0x00841b98   Section      140  faddsub.o(x$fpl$fadd)
    _fadd1                                   0x00841ba5   Thumb Code     0  faddsub.o(x$fpl$fadd)
    x$fpl$fmul                               0x00841c24   Section      176  fmul.o(x$fpl$fmul)
    x$fpl$fsub                               0x00841cd4   Section      208  faddsub.o(x$fpl$fsub)
    _fsub1                                   0x00841ce1   Thumb Code     0  faddsub.o(x$fpl$fsub)
    x$fpl$printf1                            0x00841da4   Section       16  printf1.o(x$fpl$printf1)
    x$fpl$printf2                            0x00841db4   Section       16  printf2.o(x$fpl$printf2)
    .constdata                               0x00841dc4   Section       12  system_rtl876x.o(.constdata)
    x$fpl$usenofp                            0x00841dc4   Section        0  usenofp.o(x$fpl$usenofp)
    .constdata                               0x00841dd0   Section      256  system_rtl876x.o(.constdata)
    __func__                                 0x00841dd0   Data           7  system_rtl876x.o(.constdata)
    __func__                                 0x00841dd7   Data           7  system_rtl876x.o(.constdata)
    __func__                                 0x00841dde   Data           8  system_rtl876x.o(.constdata)
    .constdata                               0x00841ed0   Section      156  rtl876x_pinmux.o(.constdata)
    .constdata                               0x00841f6c   Section      544  dis.o(.constdata)
    dis_attr_tbl                             0x00841f6c   Data         532  dis.o(.constdata)
    .constdata                               0x0084218c   Section      124  bas.o(.constdata)
    bas_attr_tbl                             0x0084218c   Data         112  bas.o(.constdata)
    .constdata                               0x00842208   Section      544  hids_rmc.o(.constdata)
    hids_report_descriptor                   0x00842208   Data          55  hids_rmc.o(.constdata)
    .constdata                               0x00842428   Section       16  vendor_service.o(.constdata)
    GATT_UUID_VENDOR_SERVICE                 0x00842428   Data          16  vendor_service.o(.constdata)
    .constdata                               0x00842438   Section      180  vendor_service.o(.constdata)
    .constdata                               0x008424ec   Section       16  atvv_service.o(.constdata)
    .constdata                               0x008424fc   Section      264  atvv_service.o(.constdata)
    .constdata                               0x00842604   Section       16  ir_service.o(.constdata)
    GATT_UUID_IR_SERVICE                     0x00842604   Data          16  ir_service.o(.constdata)
    .constdata                               0x00842614   Section      348  ir_service.o(.constdata)
    .constdata                               0x00842770   Section       16  dfu_service.o(.constdata)
    .constdata                               0x00842780   Section       12  dfu_service.o(.constdata)
    .constdata                               0x0084278c   Section       16  ota_service.o(.constdata)
    .constdata                               0x0084279c   Section      712  ota_service.o(.constdata)
    .constdata                               0x00842a64   Section       16  fms.o(.constdata)
    GATT_UUID_FMS_SERVICE                    0x00842a64   Data          16  fms.o(.constdata)
    .constdata                               0x00842a74   Section      180  fms.o(.constdata)
    .constdata                               0x00842b28   Section       29  rcu_application.o(.constdata)
    .constdata                               0x00842b45   Section       13  rcu_gap.o(.constdata)
    app_adv_data_fixed_part                  0x00842b45   Data          13  rcu_gap.o(.constdata)
    .constdata                               0x00842b52   Section       47  app_task.o(.constdata)
    __func__                                 0x00842b52   Data          14  app_task.o(.constdata)
    __func__                                 0x00842b60   Data          24  app_task.o(.constdata)
    __func__                                 0x00842b78   Data           9  app_task.o(.constdata)
    .constdata                               0x00842b81   Section       13  privacy_mgnt.o(.constdata)
    __func__                                 0x00842b81   Data          13  privacy_mgnt.o(.constdata)
    .constdata                               0x00842b8e   Section       16  loop_queue.o(.constdata)
    __func__                                 0x00842b8e   Data          16  loop_queue.o(.constdata)
    .constdata                               0x00842ba0   Section      428  key_handle.o(.constdata)
    .constdata                               0x00842d4c   Section        3  key_handle.o(.constdata)
    .constdata                               0x00842d4f   Section        8  key_handle.o(.constdata)
    .constdata                               0x00842d57   Section        3  key_handle.o(.constdata)
    .constdata                               0x00842d5a   Section       42  key_handle.o(.constdata)
    .constdata                               0x00842d84   Section        8  key_handle.o(.constdata)
    .constdata                               0x00842d8c   Section       12  key_handle.o(.constdata)
    .constdata                               0x00842d98   Section        8  key_handle.o(.constdata)
    .constdata                               0x00842da0   Section       31  voice.o(.constdata)
    __func__                                 0x00842da0   Data          31  voice.o(.constdata)
    .constdata                               0x00842dc0   Section      112  ir_protocol_nec.o(.constdata)
    .constdata                               0x00842e30   Section       40  ir_service_handle.o(.constdata)
    .constdata                               0x00842e58   Section      208  led_driver.o(.constdata)
    led_event_arr                            0x00842e58   Data         208  led_driver.o(.constdata)
    .constdata                               0x00842f28   Section       16  led_pwm_driver.o(.constdata)
    led_pwm_list                             0x00842f28   Data          16  led_pwm_driver.o(.constdata)
    .constdata                               0x00842f38   Section       36  app_custom.o(.constdata)
    .constdata                               0x00842f5c   Section      128  ddiv.o(.constdata)
    ddiv_reciptbl                            0x00842f5c   Data         128  ddiv.o(.constdata)
    .constdata                               0x00842fdc   Section       64  fdiv.o(.constdata)
    fdiv_tab                                 0x00842fdc   Data          64  fdiv.o(.constdata)
    .constdata                               0x0084301c   Section        8  _printf_wctomb.o(.constdata)
    initial_mbstate                          0x0084301c   Data           8  _printf_wctomb.o(.constdata)
    .constdata                               0x00843024   Section       40  _printf_hex_int_ll_ptr.o(.constdata)
    uc_hextab                                0x00843024   Data          20  _printf_hex_int_ll_ptr.o(.constdata)
    lc_hextab                                0x00843038   Data          20  _printf_hex_int_ll_ptr.o(.constdata)
    .constdata                               0x0084304c   Section       17  __printf_flags_ss_wp.o(.constdata)
    maptable                                 0x0084304c   Data          17  __printf_flags_ss_wp.o(.constdata)
    .constdata                               0x0084305d   Section       38  _printf_fp_hex.o(.constdata)
    lc_hextab                                0x0084305d   Data          19  _printf_fp_hex.o(.constdata)
    uc_hextab                                0x00843070   Data          19  _printf_fp_hex.o(.constdata)
    .constdata                               0x00843084   Section      148  bigflt0.o(.constdata)
    tenpwrs_x                                0x00843084   Data          60  bigflt0.o(.constdata)
    tenpwrs_i                                0x008430c0   Data          64  bigflt0.o(.constdata)
    .conststring                             0x00843118   Section      512  system_rtl876x.o(.conststring)
    .conststring                             0x00843318   Section      103  dfu_service.o(.conststring)
    .conststring                             0x00843380   Section       25  overlay_mgr.o(.conststring)
    .conststring                             0x0084339c   Section       10  app_custom.o(.conststring)
    .conststring                             0x008433a8   Section      134  frm_vpk_hal_sflash.o(.conststring)
    locale$$data                             0x00843430   Section       28  lc_numeric_c.o(locale$$data)
    __lcnum_c_name                           0x00843434   Data           2  lc_numeric_c.o(locale$$data)
    __lcnum_c_start                          0x0084343c   Data           0  lc_numeric_c.o(locale$$data)
    __lcnum_c_point                          0x00843448   Data           0  lc_numeric_c.o(locale$$data)
    __lcnum_c_thousands                      0x0084344a   Data           0  lc_numeric_c.o(locale$$data)
    __lcnum_c_grouping                       0x0084344b   Data           0  lc_numeric_c.o(locale$$data)
    locale$$data                             0x0084344c   Section      272  lc_ctype_c.o(locale$$data)
    __lcnum_c_end                            0x0084344c   Data           0  lc_numeric_c.o(locale$$data)
    __lcctype_c_name                         0x00843450   Data           2  lc_ctype_c.o(locale$$data)
    __lcctype_c_start                        0x00843458   Data           0  lc_ctype_c.o(locale$$data)
    __lcctype_c_end                          0x0084355c   Data           0  lc_ctype_c.o(locale$$data)
    .TRACE                                   0x08800000   Section      274  system_rtl876x.o(.TRACE)
    __tagsym$$used                           0x08800000   Number         0  system_rtl876x.o(.TRACE)
    format                                   0x08800000   Data          32  system_rtl876x.o(.TRACE)
    __tagsym$$used                           0x08800020   Number         0  system_rtl876x.o(.TRACE)
    format                                   0x08800020   Data          43  system_rtl876x.o(.TRACE)
    __tagsym$$used                           0x0880004c   Number         0  system_rtl876x.o(.TRACE)
    format                                   0x0880004c   Data          41  system_rtl876x.o(.TRACE)
    __tagsym$$used                           0x08800078   Number         0  system_rtl876x.o(.TRACE)
    format                                   0x08800078   Data          45  system_rtl876x.o(.TRACE)
    __tagsym$$used                           0x088000a8   Number         0  system_rtl876x.o(.TRACE)
    format                                   0x088000a8   Data          31  system_rtl876x.o(.TRACE)
    __tagsym$$used                           0x088000c8   Number         0  system_rtl876x.o(.TRACE)
    format                                   0x088000c8   Data          34  system_rtl876x.o(.TRACE)
    __tagsym$$used                           0x088000ec   Number         0  system_rtl876x.o(.TRACE)
    format                                   0x088000ec   Data          38  system_rtl876x.o(.TRACE)
    .TRACE                                   0x08800114   Section       42  rtl876x_io_dlps.o(.TRACE)
    __tagsym$$used                           0x08800114   Number         0  rtl876x_io_dlps.o(.TRACE)
    format                                   0x08800114   Data          42  rtl876x_io_dlps.o(.TRACE)
    .TRACE                                   0x08800140   Section      174  dis.o(.TRACE)
    __tagsym$$used                           0x08800140   Number         0  dis.o(.TRACE)
    format                                   0x08800140   Data          43  dis.o(.TRACE)
    __tagsym$$used                           0x0880016c   Number         0  dis.o(.TRACE)
    format                                   0x0880016c   Data          37  dis.o(.TRACE)
    __tagsym$$used                           0x08800194   Number         0  dis.o(.TRACE)
    format                                   0x08800194   Data          53  dis.o(.TRACE)
    __tagsym$$used                           0x088001cc   Number         0  dis.o(.TRACE)
    format                                   0x088001cc   Data          34  dis.o(.TRACE)
    .TRACE                                   0x088001f0   Section      222  bas.o(.TRACE)
    __tagsym$$used                           0x088001f0   Number         0  bas.o(.TRACE)
    format                                   0x088001f0   Data          48  bas.o(.TRACE)
    __tagsym$$used                           0x08800220   Number         0  bas.o(.TRACE)
    format                                   0x08800220   Data          47  bas.o(.TRACE)
    __tagsym$$used                           0x08800250   Number         0  bas.o(.TRACE)
    format                                   0x08800250   Data          42  bas.o(.TRACE)
    __tagsym$$used                           0x0880027c   Number         0  bas.o(.TRACE)
    format                                   0x0880027c   Data          48  bas.o(.TRACE)
    __tagsym$$used                           0x088002ac   Number         0  bas.o(.TRACE)
    format                                   0x088002ac   Data          34  bas.o(.TRACE)
    .TRACE                                   0x088002d0   Section      266  hids_rmc.o(.TRACE)
    __tagsym$$used                           0x088002d0   Number         0  hids_rmc.o(.TRACE)
    format                                   0x088002d0   Data          49  hids_rmc.o(.TRACE)
    __tagsym$$used                           0x08800304   Number         0  hids_rmc.o(.TRACE)
    format                                   0x08800304   Data          47  hids_rmc.o(.TRACE)
    __tagsym$$used                           0x08800334   Number         0  hids_rmc.o(.TRACE)
    format                                   0x08800334   Data          41  hids_rmc.o(.TRACE)
    __tagsym$$used                           0x08800360   Number         0  hids_rmc.o(.TRACE)
    format                                   0x08800360   Data          39  hids_rmc.o(.TRACE)
    __tagsym$$used                           0x08800388   Number         0  hids_rmc.o(.TRACE)
    format                                   0x08800388   Data          46  hids_rmc.o(.TRACE)
    __tagsym$$used                           0x088003b8   Number         0  hids_rmc.o(.TRACE)
    format                                   0x088003b8   Data          34  hids_rmc.o(.TRACE)
    .TRACE                                   0x088003dc   Section      149  vendor_service.o(.TRACE)
    __tagsym$$used                           0x088003dc   Number         0  vendor_service.o(.TRACE)
    format                                   0x088003dc   Data          49  vendor_service.o(.TRACE)
    __tagsym$$used                           0x08800410   Number         0  vendor_service.o(.TRACE)
    format                                   0x08800410   Data          55  vendor_service.o(.TRACE)
    __tagsym$$used                           0x08800448   Number         0  vendor_service.o(.TRACE)
    format                                   0x08800448   Data          41  vendor_service.o(.TRACE)
    .TRACE                                   0x08800474   Section      299  voice_service.o(.TRACE)
    __tagsym$$used                           0x08800474   Number         0  voice_service.o(.TRACE)
    format                                   0x08800474   Data          50  voice_service.o(.TRACE)
    __tagsym$$used                           0x088004a8   Number         0  voice_service.o(.TRACE)
    format                                   0x088004a8   Data          50  voice_service.o(.TRACE)
    __tagsym$$used                           0x088004dc   Number         0  voice_service.o(.TRACE)
    format                                   0x088004dc   Data          41  voice_service.o(.TRACE)
    __tagsym$$used                           0x08800508   Number         0  voice_service.o(.TRACE)
    format                                   0x08800508   Data          47  voice_service.o(.TRACE)
    __tagsym$$used                           0x08800538   Number         0  voice_service.o(.TRACE)
    format                                   0x08800538   Data          54  voice_service.o(.TRACE)
    __tagsym$$used                           0x08800570   Number         0  voice_service.o(.TRACE)
    format                                   0x08800570   Data          47  voice_service.o(.TRACE)
    .TRACE                                   0x088005a0   Section      310  atvv_service.o(.TRACE)
    __tagsym$$used                           0x088005a0   Number         0  atvv_service.o(.TRACE)
    format                                   0x088005a0   Data          48  atvv_service.o(.TRACE)
    __tagsym$$used                           0x088005d0   Number         0  atvv_service.o(.TRACE)
    format                                   0x088005d0   Data          49  atvv_service.o(.TRACE)
    __tagsym$$used                           0x08800604   Number         0  atvv_service.o(.TRACE)
    format                                   0x08800604   Data          85  atvv_service.o(.TRACE)
    __tagsym$$used                           0x0880065c   Number         0  atvv_service.o(.TRACE)
    format                                   0x0880065c   Data          40  atvv_service.o(.TRACE)
    __tagsym$$used                           0x08800684   Number         0  atvv_service.o(.TRACE)
    format                                   0x08800684   Data          46  atvv_service.o(.TRACE)
    __tagsym$$used                           0x088006b4   Number         0  atvv_service.o(.TRACE)
    format                                   0x088006b4   Data          34  atvv_service.o(.TRACE)
    .TRACE                                   0x088006d8   Section      137  ir_service.o(.TRACE)
    __tagsym$$used                           0x088006d8   Number         0  ir_service.o(.TRACE)
    format                                   0x088006d8   Data          45  ir_service.o(.TRACE)
    __tagsym$$used                           0x08800708   Number         0  ir_service.o(.TRACE)
    format                                   0x08800708   Data          51  ir_service.o(.TRACE)
    __tagsym$$used                           0x0880073c   Number         0  ir_service.o(.TRACE)
    format                                   0x0880073c   Data          37  ir_service.o(.TRACE)
    .TRACE                                   0x08800764   Section     2542  dfu_service.o(.TRACE)
    __tagsym$$used                           0x08800764   Number         0  dfu_service.o(.TRACE)
    format                                   0x08800764   Data          81  dfu_service.o(.TRACE)
    __tagsym$$used                           0x088007b8   Number         0  dfu_service.o(.TRACE)
    format                                   0x088007b8   Data          61  dfu_service.o(.TRACE)
    __tagsym$$used                           0x088007f8   Number         0  dfu_service.o(.TRACE)
    format                                   0x088007f8   Data          88  dfu_service.o(.TRACE)
    __tagsym$$used                           0x08800850   Number         0  dfu_service.o(.TRACE)
    format                                   0x08800850   Data          58  dfu_service.o(.TRACE)
    __tagsym$$used                           0x0880088c   Number         0  dfu_service.o(.TRACE)
    format                                   0x0880088c   Data          72  dfu_service.o(.TRACE)
    __tagsym$$used                           0x088008d4   Number         0  dfu_service.o(.TRACE)
    format                                   0x088008d4   Data          54  dfu_service.o(.TRACE)
    __tagsym$$used                           0x0880090c   Number         0  dfu_service.o(.TRACE)
    format                                   0x0880090c   Data          72  dfu_service.o(.TRACE)
    __tagsym$$used                           0x08800954   Number         0  dfu_service.o(.TRACE)
    format                                   0x08800954   Data          56  dfu_service.o(.TRACE)
    __tagsym$$used                           0x0880098c   Number         0  dfu_service.o(.TRACE)
    format                                   0x0880098c   Data         112  dfu_service.o(.TRACE)
    __tagsym$$used                           0x088009fc   Number         0  dfu_service.o(.TRACE)
    format                                   0x088009fc   Data          54  dfu_service.o(.TRACE)
    __tagsym$$used                           0x08800a34   Number         0  dfu_service.o(.TRACE)
    format                                   0x08800a34   Data          70  dfu_service.o(.TRACE)
    __tagsym$$used                           0x08800a7c   Number         0  dfu_service.o(.TRACE)
    format                                   0x08800a7c   Data          43  dfu_service.o(.TRACE)
    __tagsym$$used                           0x08800aa8   Number         0  dfu_service.o(.TRACE)
    format                                   0x08800aa8   Data          64  dfu_service.o(.TRACE)
    __tagsym$$used                           0x08800ae8   Number         0  dfu_service.o(.TRACE)
    format                                   0x08800ae8   Data          34  dfu_service.o(.TRACE)
    __tagsym$$used                           0x08800b0c   Number         0  dfu_service.o(.TRACE)
    format                                   0x08800b0c   Data          33  dfu_service.o(.TRACE)
    __tagsym$$used                           0x08800b30   Number         0  dfu_service.o(.TRACE)
    format                                   0x08800b30   Data         123  dfu_service.o(.TRACE)
    __tagsym$$used                           0x08800bac   Number         0  dfu_service.o(.TRACE)
    format                                   0x08800bac   Data          89  dfu_service.o(.TRACE)
    __tagsym$$used                           0x08800c08   Number         0  dfu_service.o(.TRACE)
    format                                   0x08800c08   Data          40  dfu_service.o(.TRACE)
    __tagsym$$used                           0x08800c30   Number         0  dfu_service.o(.TRACE)
    format                                   0x08800c30   Data          46  dfu_service.o(.TRACE)
    __tagsym$$used                           0x08800c60   Number         0  dfu_service.o(.TRACE)
    format                                   0x08800c60   Data          45  dfu_service.o(.TRACE)
    __tagsym$$used                           0x08800c90   Number         0  dfu_service.o(.TRACE)
    format                                   0x08800c90   Data          94  dfu_service.o(.TRACE)
    __tagsym$$used                           0x08800cf0   Number         0  dfu_service.o(.TRACE)
    format                                   0x08800cf0   Data          54  dfu_service.o(.TRACE)
    __tagsym$$used                           0x08800d28   Number         0  dfu_service.o(.TRACE)
    format                                   0x08800d28   Data          35  dfu_service.o(.TRACE)
    __tagsym$$used                           0x08800d4c   Number         0  dfu_service.o(.TRACE)
    format                                   0x08800d4c   Data          61  dfu_service.o(.TRACE)
    __tagsym$$used                           0x08800d8c   Number         0  dfu_service.o(.TRACE)
    format                                   0x08800d8c   Data          41  dfu_service.o(.TRACE)
    __tagsym$$used                           0x08800db8   Number         0  dfu_service.o(.TRACE)
    format                                   0x08800db8   Data          33  dfu_service.o(.TRACE)
    __tagsym$$used                           0x08800ddc   Number         0  dfu_service.o(.TRACE)
    format                                   0x08800ddc   Data          85  dfu_service.o(.TRACE)
    __tagsym$$used                           0x08800e34   Number         0  dfu_service.o(.TRACE)
    format                                   0x08800e34   Data          51  dfu_service.o(.TRACE)
    __tagsym$$used                           0x08800e68   Number         0  dfu_service.o(.TRACE)
    format                                   0x08800e68   Data          61  dfu_service.o(.TRACE)
    __tagsym$$used                           0x08800ea8   Number         0  dfu_service.o(.TRACE)
    format                                   0x08800ea8   Data          61  dfu_service.o(.TRACE)
    __tagsym$$used                           0x08800ee8   Number         0  dfu_service.o(.TRACE)
    format                                   0x08800ee8   Data          44  dfu_service.o(.TRACE)
    __tagsym$$used                           0x08800f14   Number         0  dfu_service.o(.TRACE)
    format                                   0x08800f14   Data          24  dfu_service.o(.TRACE)
    __tagsym$$used                           0x08800f2c   Number         0  dfu_service.o(.TRACE)
    format                                   0x08800f2c   Data          42  dfu_service.o(.TRACE)
    __tagsym$$used                           0x08800f58   Number         0  dfu_service.o(.TRACE)
    format                                   0x08800f58   Data          58  dfu_service.o(.TRACE)
    __tagsym$$used                           0x08800f94   Number         0  dfu_service.o(.TRACE)
    format                                   0x08800f94   Data         110  dfu_service.o(.TRACE)
    __tagsym$$used                           0x08801004   Number         0  dfu_service.o(.TRACE)
    format                                   0x08801004   Data         106  dfu_service.o(.TRACE)
    __tagsym$$used                           0x08801070   Number         0  dfu_service.o(.TRACE)
    format                                   0x08801070   Data         100  dfu_service.o(.TRACE)
    __tagsym$$used                           0x088010d4   Number         0  dfu_service.o(.TRACE)
    format                                   0x088010d4   Data          43  dfu_service.o(.TRACE)
    __tagsym$$used                           0x08801100   Number         0  dfu_service.o(.TRACE)
    format                                   0x08801100   Data          47  dfu_service.o(.TRACE)
    __tagsym$$used                           0x08801130   Number         0  dfu_service.o(.TRACE)
    format                                   0x08801130   Data          34  dfu_service.o(.TRACE)
    .TRACE                                   0x08801154   Section      753  ota_service.o(.TRACE)
    __tagsym$$used                           0x08801154   Number         0  ota_service.o(.TRACE)
    format                                   0x08801154   Data          65  ota_service.o(.TRACE)
    __tagsym$$used                           0x08801198   Number         0  ota_service.o(.TRACE)
    format                                   0x08801198   Data          51  ota_service.o(.TRACE)
    __tagsym$$used                           0x088011cc   Number         0  ota_service.o(.TRACE)
    format                                   0x088011cc   Data          51  ota_service.o(.TRACE)
    __tagsym$$used                           0x08801200   Number         0  ota_service.o(.TRACE)
    format                                   0x08801200   Data          49  ota_service.o(.TRACE)
    __tagsym$$used                           0x08801234   Number         0  ota_service.o(.TRACE)
    format                                   0x08801234   Data          87  ota_service.o(.TRACE)
    __tagsym$$used                           0x0880128c   Number         0  ota_service.o(.TRACE)
    format                                   0x0880128c   Data          73  ota_service.o(.TRACE)
    __tagsym$$used                           0x088012d8   Number         0  ota_service.o(.TRACE)
    format                                   0x088012d8   Data          95  ota_service.o(.TRACE)
    __tagsym$$used                           0x08801338   Number         0  ota_service.o(.TRACE)
    format                                   0x08801338   Data          61  ota_service.o(.TRACE)
    __tagsym$$used                           0x08801378   Number         0  ota_service.o(.TRACE)
    format                                   0x08801378   Data          35  ota_service.o(.TRACE)
    __tagsym$$used                           0x0880139c   Number         0  ota_service.o(.TRACE)
    format                                   0x0880139c   Data          52  ota_service.o(.TRACE)
    __tagsym$$used                           0x088013d0   Number         0  ota_service.o(.TRACE)
    format                                   0x088013d0   Data          52  ota_service.o(.TRACE)
    __tagsym$$used                           0x08801404   Number         0  ota_service.o(.TRACE)
    format                                   0x08801404   Data          27  ota_service.o(.TRACE)
    __tagsym$$used                           0x08801420   Number         0  ota_service.o(.TRACE)
    format                                   0x08801420   Data          37  ota_service.o(.TRACE)
    .TRACE                                   0x08801448   Section      174  fms.o(.TRACE)
    __tagsym$$used                           0x08801448   Number         0  fms.o(.TRACE)
    format                                   0x08801448   Data          48  fms.o(.TRACE)
    __tagsym$$used                           0x08801478   Number         0  fms.o(.TRACE)
    format                                   0x08801478   Data          42  fms.o(.TRACE)
    __tagsym$$used                           0x088014a4   Number         0  fms.o(.TRACE)
    format                                   0x088014a4   Data          48  fms.o(.TRACE)
    __tagsym$$used                           0x088014d4   Number         0  fms.o(.TRACE)
    format                                   0x088014d4   Data          34  fms.o(.TRACE)
    .TRACE                                   0x088014f8   Section      858  main.o(.TRACE)
    __tagsym$$used                           0x088014f8   Number         0  main.o(.TRACE)
    format                                   0x088014f8   Data          39  main.o(.TRACE)
    __tagsym$$used                           0x08801520   Number         0  main.o(.TRACE)
    format                                   0x08801520   Data          44  main.o(.TRACE)
    __tagsym$$used                           0x0880154c   Number         0  main.o(.TRACE)
    format                                   0x0880154c   Data          38  main.o(.TRACE)
    __tagsym$$used                           0x08801574   Number         0  main.o(.TRACE)
    format                                   0x08801574   Data          38  main.o(.TRACE)
    __tagsym$$used                           0x0880159c   Number         0  main.o(.TRACE)
    format                                   0x0880159c   Data          34  main.o(.TRACE)
    __tagsym$$used                           0x088015c0   Number         0  main.o(.TRACE)
    format                                   0x088015c0   Data          39  main.o(.TRACE)
    __tagsym$$used                           0x088015e8   Number         0  main.o(.TRACE)
    format                                   0x088015e8   Data          45  main.o(.TRACE)
    __tagsym$$used                           0x08801618   Number         0  main.o(.TRACE)
    format                                   0x08801618   Data          48  main.o(.TRACE)
    __tagsym$$used                           0x08801648   Number         0  main.o(.TRACE)
    format                                   0x08801648   Data          49  main.o(.TRACE)
    __tagsym$$used                           0x0880167c   Number         0  main.o(.TRACE)
    format                                   0x0880167c   Data          49  main.o(.TRACE)
    __tagsym$$used                           0x088016b0   Number         0  main.o(.TRACE)
    format                                   0x088016b0   Data          58  main.o(.TRACE)
    __tagsym$$used                           0x088016ec   Number         0  main.o(.TRACE)
    format                                   0x088016ec   Data          44  main.o(.TRACE)
    __tagsym$$used                           0x08801718   Number         0  main.o(.TRACE)
    format                                   0x08801718   Data          44  main.o(.TRACE)
    __tagsym$$used                           0x08801744   Number         0  main.o(.TRACE)
    format                                   0x08801744   Data          55  main.o(.TRACE)
    __tagsym$$used                           0x0880177c   Number         0  main.o(.TRACE)
    format                                   0x0880177c   Data          57  main.o(.TRACE)
    __tagsym$$used                           0x088017b8   Number         0  main.o(.TRACE)
    format                                   0x088017b8   Data          56  main.o(.TRACE)
    __tagsym$$used                           0x088017f0   Number         0  main.o(.TRACE)
    format                                   0x088017f0   Data          30  main.o(.TRACE)
    __tagsym$$used                           0x08801810   Number         0  main.o(.TRACE)
    format                                   0x08801810   Data          19  main.o(.TRACE)
    __tagsym$$used                           0x08801824   Number         0  main.o(.TRACE)
    format                                   0x08801824   Data          27  main.o(.TRACE)
    __tagsym$$used                           0x08801840   Number         0  main.o(.TRACE)
    format                                   0x08801840   Data          18  main.o(.TRACE)
    .TRACE                                   0x08801854   Section     4517  rcu_application.o(.TRACE)
    __tagsym$$used                           0x08801854   Number         0  rcu_application.o(.TRACE)
    format                                   0x08801854   Data          42  rcu_application.o(.TRACE)
    __tagsym$$used                           0x08801880   Number         0  rcu_application.o(.TRACE)
    format                                   0x08801880   Data          30  rcu_application.o(.TRACE)
    __tagsym$$used                           0x088018a0   Number         0  rcu_application.o(.TRACE)
    format                                   0x088018a0   Data          28  rcu_application.o(.TRACE)
    __tagsym$$used                           0x088018bc   Number         0  rcu_application.o(.TRACE)
    format                                   0x088018bc   Data          28  rcu_application.o(.TRACE)
    __tagsym$$used                           0x088018d8   Number         0  rcu_application.o(.TRACE)
    format                                   0x088018d8   Data          28  rcu_application.o(.TRACE)
    __tagsym$$used                           0x088018f4   Number         0  rcu_application.o(.TRACE)
    format                                   0x088018f4   Data          29  rcu_application.o(.TRACE)
    __tagsym$$used                           0x08801914   Number         0  rcu_application.o(.TRACE)
    format                                   0x08801914   Data          29  rcu_application.o(.TRACE)
    __tagsym$$used                           0x08801934   Number         0  rcu_application.o(.TRACE)
    format                                   0x08801934   Data          25  rcu_application.o(.TRACE)
    __tagsym$$used                           0x08801950   Number         0  rcu_application.o(.TRACE)
    format                                   0x08801950   Data          42  rcu_application.o(.TRACE)
    __tagsym$$used                           0x0880197c   Number         0  rcu_application.o(.TRACE)
    format                                   0x0880197c   Data          31  rcu_application.o(.TRACE)
    __tagsym$$used                           0x0880199c   Number         0  rcu_application.o(.TRACE)
    format                                   0x0880199c   Data          56  rcu_application.o(.TRACE)
    __tagsym$$used                           0x088019d4   Number         0  rcu_application.o(.TRACE)
    format                                   0x088019d4   Data          56  rcu_application.o(.TRACE)
    __tagsym$$used                           0x08801a0c   Number         0  rcu_application.o(.TRACE)
    format                                   0x08801a0c   Data          60  rcu_application.o(.TRACE)
    __tagsym$$used                           0x08801a48   Number         0  rcu_application.o(.TRACE)
    format                                   0x08801a48   Data          77  rcu_application.o(.TRACE)
    __tagsym$$used                           0x08801a98   Number         0  rcu_application.o(.TRACE)
    format                                   0x08801a98   Data          58  rcu_application.o(.TRACE)
    __tagsym$$used                           0x08801ad4   Number         0  rcu_application.o(.TRACE)
    format                                   0x08801ad4   Data          57  rcu_application.o(.TRACE)
    __tagsym$$used                           0x08801b10   Number         0  rcu_application.o(.TRACE)
    format                                   0x08801b10   Data          52  rcu_application.o(.TRACE)
    __tagsym$$used                           0x08801b44   Number         0  rcu_application.o(.TRACE)
    format                                   0x08801b44   Data          43  rcu_application.o(.TRACE)
    __tagsym$$used                           0x08801b70   Number         0  rcu_application.o(.TRACE)
    format                                   0x08801b70   Data         104  rcu_application.o(.TRACE)
    __tagsym$$used                           0x08801bd8   Number         0  rcu_application.o(.TRACE)
    format                                   0x08801bd8   Data          42  rcu_application.o(.TRACE)
    __tagsym$$used                           0x08801c04   Number         0  rcu_application.o(.TRACE)
    format                                   0x08801c04   Data          41  rcu_application.o(.TRACE)
    __tagsym$$used                           0x08801c30   Number         0  rcu_application.o(.TRACE)
    format                                   0x08801c30   Data          54  rcu_application.o(.TRACE)
    __tagsym$$used                           0x08801c68   Number         0  rcu_application.o(.TRACE)
    format                                   0x08801c68   Data          55  rcu_application.o(.TRACE)
    __tagsym$$used                           0x08801ca0   Number         0  rcu_application.o(.TRACE)
    format                                   0x08801ca0   Data          32  rcu_application.o(.TRACE)
    __tagsym$$used                           0x08801cc0   Number         0  rcu_application.o(.TRACE)
    format                                   0x08801cc0   Data          50  rcu_application.o(.TRACE)
    __tagsym$$used                           0x08801cf4   Number         0  rcu_application.o(.TRACE)
    format                                   0x08801cf4   Data          51  rcu_application.o(.TRACE)
    __tagsym$$used                           0x08801d28   Number         0  rcu_application.o(.TRACE)
    format                                   0x08801d28   Data          53  rcu_application.o(.TRACE)
    __tagsym$$used                           0x08801d60   Number         0  rcu_application.o(.TRACE)
    format                                   0x08801d60   Data          54  rcu_application.o(.TRACE)
    __tagsym$$used                           0x08801d98   Number         0  rcu_application.o(.TRACE)
    format                                   0x08801d98   Data          43  rcu_application.o(.TRACE)
    __tagsym$$used                           0x08801dc4   Number         0  rcu_application.o(.TRACE)
    format                                   0x08801dc4   Data          35  rcu_application.o(.TRACE)
    __tagsym$$used                           0x08801de8   Number         0  rcu_application.o(.TRACE)
    format                                   0x08801de8   Data          44  rcu_application.o(.TRACE)
    __tagsym$$used                           0x08801e14   Number         0  rcu_application.o(.TRACE)
    format                                   0x08801e14   Data          45  rcu_application.o(.TRACE)
    __tagsym$$used                           0x08801e44   Number         0  rcu_application.o(.TRACE)
    format                                   0x08801e44   Data          62  rcu_application.o(.TRACE)
    __tagsym$$used                           0x08801e84   Number         0  rcu_application.o(.TRACE)
    format                                   0x08801e84   Data          60  rcu_application.o(.TRACE)
    __tagsym$$used                           0x08801ec0   Number         0  rcu_application.o(.TRACE)
    format                                   0x08801ec0   Data          73  rcu_application.o(.TRACE)
    __tagsym$$used                           0x08801f0c   Number         0  rcu_application.o(.TRACE)
    format                                   0x08801f0c   Data          44  rcu_application.o(.TRACE)
    __tagsym$$used                           0x08801f38   Number         0  rcu_application.o(.TRACE)
    format                                   0x08801f38   Data          27  rcu_application.o(.TRACE)
    __tagsym$$used                           0x08801f54   Number         0  rcu_application.o(.TRACE)
    format                                   0x08801f54   Data          28  rcu_application.o(.TRACE)
    __tagsym$$used                           0x08801f70   Number         0  rcu_application.o(.TRACE)
    format                                   0x08801f70   Data          87  rcu_application.o(.TRACE)
    __tagsym$$used                           0x08801fc8   Number         0  rcu_application.o(.TRACE)
    format                                   0x08801fc8   Data          19  rcu_application.o(.TRACE)
    __tagsym$$used                           0x08801fdc   Number         0  rcu_application.o(.TRACE)
    format                                   0x08801fdc   Data          39  rcu_application.o(.TRACE)
    __tagsym$$used                           0x08802004   Number         0  rcu_application.o(.TRACE)
    format                                   0x08802004   Data          50  rcu_application.o(.TRACE)
    __tagsym$$used                           0x08802038   Number         0  rcu_application.o(.TRACE)
    format                                   0x08802038   Data          48  rcu_application.o(.TRACE)
    __tagsym$$used                           0x08802068   Number         0  rcu_application.o(.TRACE)
    format                                   0x08802068   Data          17  rcu_application.o(.TRACE)
    __tagsym$$used                           0x0880207c   Number         0  rcu_application.o(.TRACE)
    format                                   0x0880207c   Data          24  rcu_application.o(.TRACE)
    __tagsym$$used                           0x08802094   Number         0  rcu_application.o(.TRACE)
    format                                   0x08802094   Data          76  rcu_application.o(.TRACE)
    __tagsym$$used                           0x088020e0   Number         0  rcu_application.o(.TRACE)
    format                                   0x088020e0   Data          55  rcu_application.o(.TRACE)
    __tagsym$$used                           0x08802118   Number         0  rcu_application.o(.TRACE)
    format                                   0x08802118   Data          61  rcu_application.o(.TRACE)
    __tagsym$$used                           0x08802158   Number         0  rcu_application.o(.TRACE)
    format                                   0x08802158   Data         132  rcu_application.o(.TRACE)
    __tagsym$$used                           0x088021dc   Number         0  rcu_application.o(.TRACE)
    format                                   0x088021dc   Data          45  rcu_application.o(.TRACE)
    __tagsym$$used                           0x0880220c   Number         0  rcu_application.o(.TRACE)
    format                                   0x0880220c   Data          28  rcu_application.o(.TRACE)
    __tagsym$$used                           0x08802228   Number         0  rcu_application.o(.TRACE)
    format                                   0x08802228   Data          47  rcu_application.o(.TRACE)
    __tagsym$$used                           0x08802258   Number         0  rcu_application.o(.TRACE)
    format                                   0x08802258   Data          21  rcu_application.o(.TRACE)
    __tagsym$$used                           0x08802270   Number         0  rcu_application.o(.TRACE)
    format                                   0x08802270   Data          43  rcu_application.o(.TRACE)
    __tagsym$$used                           0x0880229c   Number         0  rcu_application.o(.TRACE)
    format                                   0x0880229c   Data          57  rcu_application.o(.TRACE)
    __tagsym$$used                           0x088022d8   Number         0  rcu_application.o(.TRACE)
    format                                   0x088022d8   Data         122  rcu_application.o(.TRACE)
    __tagsym$$used                           0x08802354   Number         0  rcu_application.o(.TRACE)
    format                                   0x08802354   Data          51  rcu_application.o(.TRACE)
    __tagsym$$used                           0x08802388   Number         0  rcu_application.o(.TRACE)
    format                                   0x08802388   Data          68  rcu_application.o(.TRACE)
    __tagsym$$used                           0x088023cc   Number         0  rcu_application.o(.TRACE)
    format                                   0x088023cc   Data          69  rcu_application.o(.TRACE)
    __tagsym$$used                           0x08802414   Number         0  rcu_application.o(.TRACE)
    format                                   0x08802414   Data          40  rcu_application.o(.TRACE)
    __tagsym$$used                           0x0880243c   Number         0  rcu_application.o(.TRACE)
    format                                   0x0880243c   Data          35  rcu_application.o(.TRACE)
    __tagsym$$used                           0x08802460   Number         0  rcu_application.o(.TRACE)
    format                                   0x08802460   Data          29  rcu_application.o(.TRACE)
    __tagsym$$used                           0x08802480   Number         0  rcu_application.o(.TRACE)
    format                                   0x08802480   Data          46  rcu_application.o(.TRACE)
    __tagsym$$used                           0x088024b0   Number         0  rcu_application.o(.TRACE)
    format                                   0x088024b0   Data          49  rcu_application.o(.TRACE)
    __tagsym$$used                           0x088024e4   Number         0  rcu_application.o(.TRACE)
    format                                   0x088024e4   Data          45  rcu_application.o(.TRACE)
    __tagsym$$used                           0x08802514   Number         0  rcu_application.o(.TRACE)
    format                                   0x08802514   Data          29  rcu_application.o(.TRACE)
    __tagsym$$used                           0x08802534   Number         0  rcu_application.o(.TRACE)
    format                                   0x08802534   Data          49  rcu_application.o(.TRACE)
    __tagsym$$used                           0x08802568   Number         0  rcu_application.o(.TRACE)
    format                                   0x08802568   Data          45  rcu_application.o(.TRACE)
    __tagsym$$used                           0x08802598   Number         0  rcu_application.o(.TRACE)
    format                                   0x08802598   Data          63  rcu_application.o(.TRACE)
    __tagsym$$used                           0x088025d8   Number         0  rcu_application.o(.TRACE)
    format                                   0x088025d8   Data          49  rcu_application.o(.TRACE)
    __tagsym$$used                           0x0880260c   Number         0  rcu_application.o(.TRACE)
    format                                   0x0880260c   Data          55  rcu_application.o(.TRACE)
    __tagsym$$used                           0x08802644   Number         0  rcu_application.o(.TRACE)
    format                                   0x08802644   Data          63  rcu_application.o(.TRACE)
    __tagsym$$used                           0x08802684   Number         0  rcu_application.o(.TRACE)
    format                                   0x08802684   Data          64  rcu_application.o(.TRACE)
    __tagsym$$used                           0x088026c4   Number         0  rcu_application.o(.TRACE)
    format                                   0x088026c4   Data          93  rcu_application.o(.TRACE)
    __tagsym$$used                           0x08802724   Number         0  rcu_application.o(.TRACE)
    format                                   0x08802724   Data          45  rcu_application.o(.TRACE)
    __tagsym$$used                           0x08802754   Number         0  rcu_application.o(.TRACE)
    format                                   0x08802754   Data          38  rcu_application.o(.TRACE)
    __tagsym$$used                           0x0880277c   Number         0  rcu_application.o(.TRACE)
    format                                   0x0880277c   Data          32  rcu_application.o(.TRACE)
    __tagsym$$used                           0x0880279c   Number         0  rcu_application.o(.TRACE)
    format                                   0x0880279c   Data          30  rcu_application.o(.TRACE)
    __tagsym$$used                           0x088027bc   Number         0  rcu_application.o(.TRACE)
    format                                   0x088027bc   Data          81  rcu_application.o(.TRACE)
    __tagsym$$used                           0x08802810   Number         0  rcu_application.o(.TRACE)
    format                                   0x08802810   Data          42  rcu_application.o(.TRACE)
    __tagsym$$used                           0x0880283c   Number         0  rcu_application.o(.TRACE)
    format                                   0x0880283c   Data          58  rcu_application.o(.TRACE)
    __tagsym$$used                           0x08802878   Number         0  rcu_application.o(.TRACE)
    format                                   0x08802878   Data          48  rcu_application.o(.TRACE)
    __tagsym$$used                           0x088028a8   Number         0  rcu_application.o(.TRACE)
    format                                   0x088028a8   Data          58  rcu_application.o(.TRACE)
    __tagsym$$used                           0x088028e4   Number         0  rcu_application.o(.TRACE)
    format                                   0x088028e4   Data          42  rcu_application.o(.TRACE)
    __tagsym$$used                           0x08802910   Number         0  rcu_application.o(.TRACE)
    format                                   0x08802910   Data          44  rcu_application.o(.TRACE)
    __tagsym$$used                           0x0880293c   Number         0  rcu_application.o(.TRACE)
    format                                   0x0880293c   Data          44  rcu_application.o(.TRACE)
    __tagsym$$used                           0x08802968   Number         0  rcu_application.o(.TRACE)
    format                                   0x08802968   Data          33  rcu_application.o(.TRACE)
    __tagsym$$used                           0x0880298c   Number         0  rcu_application.o(.TRACE)
    format                                   0x0880298c   Data          53  rcu_application.o(.TRACE)
    __tagsym$$used                           0x088029c4   Number         0  rcu_application.o(.TRACE)
    format                                   0x088029c4   Data          53  rcu_application.o(.TRACE)
    .TRACE                                   0x088029fc   Section     1756  rcu_gap.o(.TRACE)
    __tagsym$$used                           0x088029fc   Number         0  rcu_gap.o(.TRACE)
    format                                   0x088029fc   Data          19  rcu_gap.o(.TRACE)
    __tagsym$$used                           0x08802a10   Number         0  rcu_gap.o(.TRACE)
    format                                   0x08802a10   Data          52  rcu_gap.o(.TRACE)
    __tagsym$$used                           0x08802a44   Number         0  rcu_gap.o(.TRACE)
    format                                   0x08802a44   Data          43  rcu_gap.o(.TRACE)
    __tagsym$$used                           0x08802a70   Number         0  rcu_gap.o(.TRACE)
    format                                   0x08802a70   Data          47  rcu_gap.o(.TRACE)
    __tagsym$$used                           0x08802aa0   Number         0  rcu_gap.o(.TRACE)
    format                                   0x08802aa0   Data          37  rcu_gap.o(.TRACE)
    __tagsym$$used                           0x08802ac8   Number         0  rcu_gap.o(.TRACE)
    format                                   0x08802ac8   Data          34  rcu_gap.o(.TRACE)
    __tagsym$$used                           0x08802aec   Number         0  rcu_gap.o(.TRACE)
    format                                   0x08802aec   Data          43  rcu_gap.o(.TRACE)
    __tagsym$$used                           0x08802b18   Number         0  rcu_gap.o(.TRACE)
    format                                   0x08802b18   Data          47  rcu_gap.o(.TRACE)
    __tagsym$$used                           0x08802b48   Number         0  rcu_gap.o(.TRACE)
    format                                   0x08802b48   Data          37  rcu_gap.o(.TRACE)
    __tagsym$$used                           0x08802b70   Number         0  rcu_gap.o(.TRACE)
    format                                   0x08802b70   Data          34  rcu_gap.o(.TRACE)
    __tagsym$$used                           0x08802b94   Number         0  rcu_gap.o(.TRACE)
    format                                   0x08802b94   Data          43  rcu_gap.o(.TRACE)
    __tagsym$$used                           0x08802bc0   Number         0  rcu_gap.o(.TRACE)
    format                                   0x08802bc0   Data          47  rcu_gap.o(.TRACE)
    __tagsym$$used                           0x08802bf0   Number         0  rcu_gap.o(.TRACE)
    format                                   0x08802bf0   Data          40  rcu_gap.o(.TRACE)
    __tagsym$$used                           0x08802c18   Number         0  rcu_gap.o(.TRACE)
    format                                   0x08802c18   Data          37  rcu_gap.o(.TRACE)
    __tagsym$$used                           0x08802c40   Number         0  rcu_gap.o(.TRACE)
    format                                   0x08802c40   Data          43  rcu_gap.o(.TRACE)
    __tagsym$$used                           0x08802c6c   Number         0  rcu_gap.o(.TRACE)
    format                                   0x08802c6c   Data          45  rcu_gap.o(.TRACE)
    __tagsym$$used                           0x08802c9c   Number         0  rcu_gap.o(.TRACE)
    format                                   0x08802c9c   Data          42  rcu_gap.o(.TRACE)
    __tagsym$$used                           0x08802cc8   Number         0  rcu_gap.o(.TRACE)
    format                                   0x08802cc8   Data          54  rcu_gap.o(.TRACE)
    __tagsym$$used                           0x08802d00   Number         0  rcu_gap.o(.TRACE)
    format                                   0x08802d00   Data          43  rcu_gap.o(.TRACE)
    __tagsym$$used                           0x08802d2c   Number         0  rcu_gap.o(.TRACE)
    format                                   0x08802d2c   Data          47  rcu_gap.o(.TRACE)
    __tagsym$$used                           0x08802d5c   Number         0  rcu_gap.o(.TRACE)
    format                                   0x08802d5c   Data          66  rcu_gap.o(.TRACE)
    __tagsym$$used                           0x08802da0   Number         0  rcu_gap.o(.TRACE)
    format                                   0x08802da0   Data          39  rcu_gap.o(.TRACE)
    __tagsym$$used                           0x08802dc8   Number         0  rcu_gap.o(.TRACE)
    format                                   0x08802dc8   Data          52  rcu_gap.o(.TRACE)
    __tagsym$$used                           0x08802dfc   Number         0  rcu_gap.o(.TRACE)
    format                                   0x08802dfc   Data          37  rcu_gap.o(.TRACE)
    __tagsym$$used                           0x08802e24   Number         0  rcu_gap.o(.TRACE)
    format                                   0x08802e24   Data          43  rcu_gap.o(.TRACE)
    __tagsym$$used                           0x08802e50   Number         0  rcu_gap.o(.TRACE)
    format                                   0x08802e50   Data          40  rcu_gap.o(.TRACE)
    __tagsym$$used                           0x08802e78   Number         0  rcu_gap.o(.TRACE)
    format                                   0x08802e78   Data          40  rcu_gap.o(.TRACE)
    __tagsym$$used                           0x08802ea0   Number         0  rcu_gap.o(.TRACE)
    format                                   0x08802ea0   Data          46  rcu_gap.o(.TRACE)
    __tagsym$$used                           0x08802ed0   Number         0  rcu_gap.o(.TRACE)
    format                                   0x08802ed0   Data          43  rcu_gap.o(.TRACE)
    __tagsym$$used                           0x08802efc   Number         0  rcu_gap.o(.TRACE)
    format                                   0x08802efc   Data          40  rcu_gap.o(.TRACE)
    __tagsym$$used                           0x08802f24   Number         0  rcu_gap.o(.TRACE)
    format                                   0x08802f24   Data          53  rcu_gap.o(.TRACE)
    __tagsym$$used                           0x08802f5c   Number         0  rcu_gap.o(.TRACE)
    format                                   0x08802f5c   Data          47  rcu_gap.o(.TRACE)
    __tagsym$$used                           0x08802f8c   Number         0  rcu_gap.o(.TRACE)
    format                                   0x08802f8c   Data          41  rcu_gap.o(.TRACE)
    __tagsym$$used                           0x08802fb8   Number         0  rcu_gap.o(.TRACE)
    format                                   0x08802fb8   Data          66  rcu_gap.o(.TRACE)
    __tagsym$$used                           0x08802ffc   Number         0  rcu_gap.o(.TRACE)
    format                                   0x08802ffc   Data          60  rcu_gap.o(.TRACE)
    __tagsym$$used                           0x08803038   Number         0  rcu_gap.o(.TRACE)
    format                                   0x08803038   Data          53  rcu_gap.o(.TRACE)
    __tagsym$$used                           0x08803070   Number         0  rcu_gap.o(.TRACE)
    format                                   0x08803070   Data          51  rcu_gap.o(.TRACE)
    __tagsym$$used                           0x088030a4   Number         0  rcu_gap.o(.TRACE)
    format                                   0x088030a4   Data          52  rcu_gap.o(.TRACE)
    .TRACE                                   0x088030d8   Section      742  swtimer.o(.TRACE)
    __tagsym$$used                           0x088030d8   Number         0  swtimer.o(.TRACE)
    format                                   0x088030d8   Data          43  swtimer.o(.TRACE)
    __tagsym$$used                           0x08803104   Number         0  swtimer.o(.TRACE)
    format                                   0x08803104   Data          44  swtimer.o(.TRACE)
    __tagsym$$used                           0x08803130   Number         0  swtimer.o(.TRACE)
    format                                   0x08803130   Data          46  swtimer.o(.TRACE)
    __tagsym$$used                           0x08803160   Number         0  swtimer.o(.TRACE)
    format                                   0x08803160   Data          56  swtimer.o(.TRACE)
    __tagsym$$used                           0x08803198   Number         0  swtimer.o(.TRACE)
    format                                   0x08803198   Data          48  swtimer.o(.TRACE)
    __tagsym$$used                           0x088031c8   Number         0  swtimer.o(.TRACE)
    format                                   0x088031c8   Data          68  swtimer.o(.TRACE)
    __tagsym$$used                           0x0880320c   Number         0  swtimer.o(.TRACE)
    format                                   0x0880320c   Data          41  swtimer.o(.TRACE)
    __tagsym$$used                           0x08803238   Number         0  swtimer.o(.TRACE)
    format                                   0x08803238   Data          53  swtimer.o(.TRACE)
    __tagsym$$used                           0x08803270   Number         0  swtimer.o(.TRACE)
    format                                   0x08803270   Data          55  swtimer.o(.TRACE)
    __tagsym$$used                           0x088032a8   Number         0  swtimer.o(.TRACE)
    format                                   0x088032a8   Data          67  swtimer.o(.TRACE)
    __tagsym$$used                           0x088032ec   Number         0  swtimer.o(.TRACE)
    format                                   0x088032ec   Data          46  swtimer.o(.TRACE)
    __tagsym$$used                           0x0880331c   Number         0  swtimer.o(.TRACE)
    format                                   0x0880331c   Data          56  swtimer.o(.TRACE)
    __tagsym$$used                           0x08803354   Number         0  swtimer.o(.TRACE)
    format                                   0x08803354   Data          49  swtimer.o(.TRACE)
    __tagsym$$used                           0x08803388   Number         0  swtimer.o(.TRACE)
    format                                   0x08803388   Data          54  swtimer.o(.TRACE)
    .TRACE                                   0x088033c0   Section       56  app_task.o(.TRACE)
    __tagsym$$used                           0x088033c0   Number         0  app_task.o(.TRACE)
    format                                   0x088033c0   Data          27  app_task.o(.TRACE)
    __tagsym$$used                           0x088033dc   Number         0  app_task.o(.TRACE)
    format                                   0x088033dc   Data          28  app_task.o(.TRACE)
    .TRACE                                   0x088033f8   Section       58  reset_watch_dog_timer.o(.TRACE)
    __tagsym$$used                           0x088033f8   Number         0  reset_watch_dog_timer.o(.TRACE)
    format                                   0x088033f8   Data          58  reset_watch_dog_timer.o(.TRACE)
    .TRACE                                   0x08803434   Section     1455  privacy_mgnt.o(.TRACE)
    __tagsym$$used                           0x08803434   Number         0  privacy_mgnt.o(.TRACE)
    format                                   0x08803434   Data          48  privacy_mgnt.o(.TRACE)
    __tagsym$$used                           0x08803464   Number         0  privacy_mgnt.o(.TRACE)
    format                                   0x08803464   Data          40  privacy_mgnt.o(.TRACE)
    __tagsym$$used                           0x0880348c   Number         0  privacy_mgnt.o(.TRACE)
    format                                   0x0880348c   Data          22  privacy_mgnt.o(.TRACE)
    __tagsym$$used                           0x088034a4   Number         0  privacy_mgnt.o(.TRACE)
    format                                   0x088034a4   Data          19  privacy_mgnt.o(.TRACE)
    __tagsym$$used                           0x088034b8   Number         0  privacy_mgnt.o(.TRACE)
    format                                   0x088034b8   Data          36  privacy_mgnt.o(.TRACE)
    __tagsym$$used                           0x088034dc   Number         0  privacy_mgnt.o(.TRACE)
    format                                   0x088034dc   Data          40  privacy_mgnt.o(.TRACE)
    __tagsym$$used                           0x08803504   Number         0  privacy_mgnt.o(.TRACE)
    format                                   0x08803504   Data          62  privacy_mgnt.o(.TRACE)
    __tagsym$$used                           0x08803544   Number         0  privacy_mgnt.o(.TRACE)
    format                                   0x08803544   Data          39  privacy_mgnt.o(.TRACE)
    __tagsym$$used                           0x0880356c   Number         0  privacy_mgnt.o(.TRACE)
    format                                   0x0880356c   Data          42  privacy_mgnt.o(.TRACE)
    __tagsym$$used                           0x08803598   Number         0  privacy_mgnt.o(.TRACE)
    format                                   0x08803598   Data          65  privacy_mgnt.o(.TRACE)
    __tagsym$$used                           0x088035dc   Number         0  privacy_mgnt.o(.TRACE)
    format                                   0x088035dc   Data          42  privacy_mgnt.o(.TRACE)
    __tagsym$$used                           0x08803608   Number         0  privacy_mgnt.o(.TRACE)
    format                                   0x08803608   Data          50  privacy_mgnt.o(.TRACE)
    __tagsym$$used                           0x0880363c   Number         0  privacy_mgnt.o(.TRACE)
    format                                   0x0880363c   Data          55  privacy_mgnt.o(.TRACE)
    __tagsym$$used                           0x08803674   Number         0  privacy_mgnt.o(.TRACE)
    format                                   0x08803674   Data          51  privacy_mgnt.o(.TRACE)
    __tagsym$$used                           0x088036a8   Number         0  privacy_mgnt.o(.TRACE)
    format                                   0x088036a8   Data          59  privacy_mgnt.o(.TRACE)
    __tagsym$$used                           0x088036e4   Number         0  privacy_mgnt.o(.TRACE)
    format                                   0x088036e4   Data          51  privacy_mgnt.o(.TRACE)
    __tagsym$$used                           0x08803718   Number         0  privacy_mgnt.o(.TRACE)
    format                                   0x08803718   Data          59  privacy_mgnt.o(.TRACE)
    __tagsym$$used                           0x08803754   Number         0  privacy_mgnt.o(.TRACE)
    format                                   0x08803754   Data          62  privacy_mgnt.o(.TRACE)
    __tagsym$$used                           0x08803794   Number         0  privacy_mgnt.o(.TRACE)
    format                                   0x08803794   Data          50  privacy_mgnt.o(.TRACE)
    __tagsym$$used                           0x088037c8   Number         0  privacy_mgnt.o(.TRACE)
    format                                   0x088037c8   Data          56  privacy_mgnt.o(.TRACE)
    __tagsym$$used                           0x08803800   Number         0  privacy_mgnt.o(.TRACE)
    format                                   0x08803800   Data          76  privacy_mgnt.o(.TRACE)
    __tagsym$$used                           0x0880384c   Number         0  privacy_mgnt.o(.TRACE)
    format                                   0x0880384c   Data          91  privacy_mgnt.o(.TRACE)
    __tagsym$$used                           0x088038a8   Number         0  privacy_mgnt.o(.TRACE)
    format                                   0x088038a8   Data          48  privacy_mgnt.o(.TRACE)
    __tagsym$$used                           0x088038d8   Number         0  privacy_mgnt.o(.TRACE)
    format                                   0x088038d8   Data          53  privacy_mgnt.o(.TRACE)
    __tagsym$$used                           0x08803910   Number         0  privacy_mgnt.o(.TRACE)
    format                                   0x08803910   Data          73  privacy_mgnt.o(.TRACE)
    __tagsym$$used                           0x0880395c   Number         0  privacy_mgnt.o(.TRACE)
    format                                   0x0880395c   Data          66  privacy_mgnt.o(.TRACE)
    __tagsym$$used                           0x088039a0   Number         0  privacy_mgnt.o(.TRACE)
    format                                   0x088039a0   Data          67  privacy_mgnt.o(.TRACE)
    .TRACE                                   0x088039e4   Section      757  rcu_dtm_app.o(.TRACE)
    __tagsym$$used                           0x088039e4   Number         0  rcu_dtm_app.o(.TRACE)
    format                                   0x088039e4   Data          32  rcu_dtm_app.o(.TRACE)
    __tagsym$$used                           0x08803a04   Number         0  rcu_dtm_app.o(.TRACE)
    format                                   0x08803a04   Data          56  rcu_dtm_app.o(.TRACE)
    __tagsym$$used                           0x08803a3c   Number         0  rcu_dtm_app.o(.TRACE)
    format                                   0x08803a3c   Data          57  rcu_dtm_app.o(.TRACE)
    __tagsym$$used                           0x08803a78   Number         0  rcu_dtm_app.o(.TRACE)
    format                                   0x08803a78   Data          52  rcu_dtm_app.o(.TRACE)
    __tagsym$$used                           0x08803aac   Number         0  rcu_dtm_app.o(.TRACE)
    format                                   0x08803aac   Data          71  rcu_dtm_app.o(.TRACE)
    __tagsym$$used                           0x08803af4   Number         0  rcu_dtm_app.o(.TRACE)
    format                                   0x08803af4   Data          55  rcu_dtm_app.o(.TRACE)
    __tagsym$$used                           0x08803b2c   Number         0  rcu_dtm_app.o(.TRACE)
    format                                   0x08803b2c   Data          29  rcu_dtm_app.o(.TRACE)
    __tagsym$$used                           0x08803b4c   Number         0  rcu_dtm_app.o(.TRACE)
    format                                   0x08803b4c   Data          34  rcu_dtm_app.o(.TRACE)
    __tagsym$$used                           0x08803b70   Number         0  rcu_dtm_app.o(.TRACE)
    format                                   0x08803b70   Data          20  rcu_dtm_app.o(.TRACE)
    __tagsym$$used                           0x08803b84   Number         0  rcu_dtm_app.o(.TRACE)
    format                                   0x08803b84   Data          20  rcu_dtm_app.o(.TRACE)
    __tagsym$$used                           0x08803b98   Number         0  rcu_dtm_app.o(.TRACE)
    format                                   0x08803b98   Data          32  rcu_dtm_app.o(.TRACE)
    __tagsym$$used                           0x08803bb8   Number         0  rcu_dtm_app.o(.TRACE)
    format                                   0x08803bb8   Data          45  rcu_dtm_app.o(.TRACE)
    __tagsym$$used                           0x08803be8   Number         0  rcu_dtm_app.o(.TRACE)
    format                                   0x08803be8   Data          45  rcu_dtm_app.o(.TRACE)
    __tagsym$$used                           0x08803c18   Number         0  rcu_dtm_app.o(.TRACE)
    format                                   0x08803c18   Data          45  rcu_dtm_app.o(.TRACE)
    __tagsym$$used                           0x08803c48   Number         0  rcu_dtm_app.o(.TRACE)
    format                                   0x08803c48   Data          45  rcu_dtm_app.o(.TRACE)
    __tagsym$$used                           0x08803c78   Number         0  rcu_dtm_app.o(.TRACE)
    format                                   0x08803c78   Data          51  rcu_dtm_app.o(.TRACE)
    __tagsym$$used                           0x08803cac   Number         0  rcu_dtm_app.o(.TRACE)
    format                                   0x08803cac   Data          45  rcu_dtm_app.o(.TRACE)
    .TRACE                                   0x08803cdc   Section       83  rcu_link_mgr.o(.TRACE)
    __tagsym$$used                           0x08803cdc   Number         0  rcu_link_mgr.o(.TRACE)
    format                                   0x08803cdc   Data          34  rcu_link_mgr.o(.TRACE)
    __tagsym$$used                           0x08803d00   Number         0  rcu_link_mgr.o(.TRACE)
    format                                   0x08803d00   Data          47  rcu_link_mgr.o(.TRACE)
    .TRACE                                   0x08803d30   Section      223  rtc_driver.o(.TRACE)
    __tagsym$$used                           0x08803d30   Number         0  rtc_driver.o(.TRACE)
    format                                   0x08803d30   Data          30  rtc_driver.o(.TRACE)
    __tagsym$$used                           0x08803d50   Number         0  rtc_driver.o(.TRACE)
    format                                   0x08803d50   Data          32  rtc_driver.o(.TRACE)
    __tagsym$$used                           0x08803d70   Number         0  rtc_driver.o(.TRACE)
    format                                   0x08803d70   Data          35  rtc_driver.o(.TRACE)
    __tagsym$$used                           0x08803d94   Number         0  rtc_driver.o(.TRACE)
    format                                   0x08803d94   Data          60  rtc_driver.o(.TRACE)
    __tagsym$$used                           0x08803dd0   Number         0  rtc_driver.o(.TRACE)
    format                                   0x08803dd0   Data          29  rtc_driver.o(.TRACE)
    __tagsym$$used                           0x08803df0   Number         0  rtc_driver.o(.TRACE)
    format                                   0x08803df0   Data          31  rtc_driver.o(.TRACE)
    .TRACE                                   0x08803e10   Section     1004  dfu_flash.o(.TRACE)
    __tagsym$$used                           0x08803e10   Number         0  dfu_flash.o(.TRACE)
    format                                   0x08803e10   Data          60  dfu_flash.o(.TRACE)
    __tagsym$$used                           0x08803e4c   Number         0  dfu_flash.o(.TRACE)
    format                                   0x08803e4c   Data          59  dfu_flash.o(.TRACE)
    __tagsym$$used                           0x08803e88   Number         0  dfu_flash.o(.TRACE)
    format                                   0x08803e88   Data          72  dfu_flash.o(.TRACE)
    __tagsym$$used                           0x08803ed0   Number         0  dfu_flash.o(.TRACE)
    format                                   0x08803ed0   Data          78  dfu_flash.o(.TRACE)
    __tagsym$$used                           0x08803f20   Number         0  dfu_flash.o(.TRACE)
    format                                   0x08803f20   Data          41  dfu_flash.o(.TRACE)
    __tagsym$$used                           0x08803f4c   Number         0  dfu_flash.o(.TRACE)
    format                                   0x08803f4c   Data          33  dfu_flash.o(.TRACE)
    __tagsym$$used                           0x08803f70   Number         0  dfu_flash.o(.TRACE)
    format                                   0x08803f70   Data          30  dfu_flash.o(.TRACE)
    __tagsym$$used                           0x08803f90   Number         0  dfu_flash.o(.TRACE)
    format                                   0x08803f90   Data          34  dfu_flash.o(.TRACE)
    __tagsym$$used                           0x08803fb4   Number         0  dfu_flash.o(.TRACE)
    format                                   0x08803fb4   Data          43  dfu_flash.o(.TRACE)
    __tagsym$$used                           0x08803fe0   Number         0  dfu_flash.o(.TRACE)
    format                                   0x08803fe0   Data          43  dfu_flash.o(.TRACE)
    __tagsym$$used                           0x0880400c   Number         0  dfu_flash.o(.TRACE)
    format                                   0x0880400c   Data          77  dfu_flash.o(.TRACE)
    __tagsym$$used                           0x0880405c   Number         0  dfu_flash.o(.TRACE)
    format                                   0x0880405c   Data          37  dfu_flash.o(.TRACE)
    __tagsym$$used                           0x08804084   Number         0  dfu_flash.o(.TRACE)
    format                                   0x08804084   Data          45  dfu_flash.o(.TRACE)
    __tagsym$$used                           0x088040b4   Number         0  dfu_flash.o(.TRACE)
    format                                   0x088040b4   Data          49  dfu_flash.o(.TRACE)
    __tagsym$$used                           0x088040e8   Number         0  dfu_flash.o(.TRACE)
    format                                   0x088040e8   Data          41  dfu_flash.o(.TRACE)
    __tagsym$$used                           0x08804114   Number         0  dfu_flash.o(.TRACE)
    format                                   0x08804114   Data          54  dfu_flash.o(.TRACE)
    __tagsym$$used                           0x0880414c   Number         0  dfu_flash.o(.TRACE)
    format                                   0x0880414c   Data          72  dfu_flash.o(.TRACE)
    __tagsym$$used                           0x08804194   Number         0  dfu_flash.o(.TRACE)
    format                                   0x08804194   Data          28  dfu_flash.o(.TRACE)
    __tagsym$$used                           0x088041b0   Number         0  dfu_flash.o(.TRACE)
    format                                   0x088041b0   Data          76  dfu_flash.o(.TRACE)
    .TRACE                                   0x088041fc   Section      312  keyscan_driver.o(.TRACE)
    __tagsym$$used                           0x088041fc   Number         0  keyscan_driver.o(.TRACE)
    format                                   0x088041fc   Data          61  keyscan_driver.o(.TRACE)
    __tagsym$$used                           0x0880423c   Number         0  keyscan_driver.o(.TRACE)
    format                                   0x0880423c   Data          74  keyscan_driver.o(.TRACE)
    __tagsym$$used                           0x08804288   Number         0  keyscan_driver.o(.TRACE)
    format                                   0x08804288   Data          43  keyscan_driver.o(.TRACE)
    __tagsym$$used                           0x088042b4   Number         0  keyscan_driver.o(.TRACE)
    format                                   0x088042b4   Data          81  keyscan_driver.o(.TRACE)
    __tagsym$$used                           0x08804308   Number         0  keyscan_driver.o(.TRACE)
    format                                   0x08804308   Data          44  keyscan_driver.o(.TRACE)
    .TRACE                                   0x08804334   Section     2640  key_handle.o(.TRACE)
    __tagsym$$used                           0x08804334   Number         0  key_handle.o(.TRACE)
    format                                   0x08804334   Data          71  key_handle.o(.TRACE)
    __tagsym$$used                           0x0880437c   Number         0  key_handle.o(.TRACE)
    format                                   0x0880437c   Data          68  key_handle.o(.TRACE)
    __tagsym$$used                           0x088043c0   Number         0  key_handle.o(.TRACE)
    format                                   0x088043c0   Data          71  key_handle.o(.TRACE)
    __tagsym$$used                           0x08804408   Number         0  key_handle.o(.TRACE)
    format                                   0x08804408   Data          59  key_handle.o(.TRACE)
    __tagsym$$used                           0x08804444   Number         0  key_handle.o(.TRACE)
    format                                   0x08804444   Data          62  key_handle.o(.TRACE)
    __tagsym$$used                           0x08804484   Number         0  key_handle.o(.TRACE)
    format                                   0x08804484   Data          74  key_handle.o(.TRACE)
    __tagsym$$used                           0x088044d0   Number         0  key_handle.o(.TRACE)
    format                                   0x088044d0   Data          74  key_handle.o(.TRACE)
    __tagsym$$used                           0x0880451c   Number         0  key_handle.o(.TRACE)
    format                                   0x0880451c   Data          58  key_handle.o(.TRACE)
    __tagsym$$used                           0x08804558   Number         0  key_handle.o(.TRACE)
    format                                   0x08804558   Data          85  key_handle.o(.TRACE)
    __tagsym$$used                           0x088045b0   Number         0  key_handle.o(.TRACE)
    format                                   0x088045b0   Data          90  key_handle.o(.TRACE)
    __tagsym$$used                           0x0880460c   Number         0  key_handle.o(.TRACE)
    format                                   0x0880460c   Data          80  key_handle.o(.TRACE)
    __tagsym$$used                           0x0880465c   Number         0  key_handle.o(.TRACE)
    format                                   0x0880465c   Data          92  key_handle.o(.TRACE)
    __tagsym$$used                           0x088046b8   Number         0  key_handle.o(.TRACE)
    format                                   0x088046b8   Data          69  key_handle.o(.TRACE)
    __tagsym$$used                           0x08804700   Number         0  key_handle.o(.TRACE)
    format                                   0x08804700   Data          47  key_handle.o(.TRACE)
    __tagsym$$used                           0x08804730   Number         0  key_handle.o(.TRACE)
    format                                   0x08804730   Data          53  key_handle.o(.TRACE)
    __tagsym$$used                           0x08804768   Number         0  key_handle.o(.TRACE)
    format                                   0x08804768   Data          26  key_handle.o(.TRACE)
    __tagsym$$used                           0x08804784   Number         0  key_handle.o(.TRACE)
    format                                   0x08804784   Data          25  key_handle.o(.TRACE)
    __tagsym$$used                           0x088047a0   Number         0  key_handle.o(.TRACE)
    format                                   0x088047a0   Data          68  key_handle.o(.TRACE)
    __tagsym$$used                           0x088047e4   Number         0  key_handle.o(.TRACE)
    format                                   0x088047e4   Data          84  key_handle.o(.TRACE)
    __tagsym$$used                           0x08804838   Number         0  key_handle.o(.TRACE)
    format                                   0x08804838   Data          66  key_handle.o(.TRACE)
    __tagsym$$used                           0x0880487c   Number         0  key_handle.o(.TRACE)
    format                                   0x0880487c   Data          65  key_handle.o(.TRACE)
    __tagsym$$used                           0x088048c0   Number         0  key_handle.o(.TRACE)
    format                                   0x088048c0   Data          73  key_handle.o(.TRACE)
    __tagsym$$used                           0x0880490c   Number         0  key_handle.o(.TRACE)
    format                                   0x0880490c   Data          66  key_handle.o(.TRACE)
    __tagsym$$used                           0x08804950   Number         0  key_handle.o(.TRACE)
    format                                   0x08804950   Data          36  key_handle.o(.TRACE)
    __tagsym$$used                           0x08804974   Number         0  key_handle.o(.TRACE)
    format                                   0x08804974   Data          52  key_handle.o(.TRACE)
    __tagsym$$used                           0x088049a8   Number         0  key_handle.o(.TRACE)
    format                                   0x088049a8   Data          48  key_handle.o(.TRACE)
    __tagsym$$used                           0x088049d8   Number         0  key_handle.o(.TRACE)
    format                                   0x088049d8   Data          38  key_handle.o(.TRACE)
    __tagsym$$used                           0x08804a00   Number         0  key_handle.o(.TRACE)
    format                                   0x08804a00   Data          70  key_handle.o(.TRACE)
    __tagsym$$used                           0x08804a48   Number         0  key_handle.o(.TRACE)
    format                                   0x08804a48   Data          76  key_handle.o(.TRACE)
    __tagsym$$used                           0x08804a94   Number         0  key_handle.o(.TRACE)
    format                                   0x08804a94   Data          69  key_handle.o(.TRACE)
    __tagsym$$used                           0x08804adc   Number         0  key_handle.o(.TRACE)
    format                                   0x08804adc   Data          88  key_handle.o(.TRACE)
    __tagsym$$used                           0x08804b34   Number         0  key_handle.o(.TRACE)
    format                                   0x08804b34   Data          89  key_handle.o(.TRACE)
    __tagsym$$used                           0x08804b90   Number         0  key_handle.o(.TRACE)
    format                                   0x08804b90   Data          75  key_handle.o(.TRACE)
    __tagsym$$used                           0x08804bdc   Number         0  key_handle.o(.TRACE)
    format                                   0x08804bdc   Data          68  key_handle.o(.TRACE)
    __tagsym$$used                           0x08804c20   Number         0  key_handle.o(.TRACE)
    format                                   0x08804c20   Data          75  key_handle.o(.TRACE)
    __tagsym$$used                           0x08804c6c   Number         0  key_handle.o(.TRACE)
    format                                   0x08804c6c   Data          82  key_handle.o(.TRACE)
    __tagsym$$used                           0x08804cc0   Number         0  key_handle.o(.TRACE)
    format                                   0x08804cc0   Data          28  key_handle.o(.TRACE)
    __tagsym$$used                           0x08804cdc   Number         0  key_handle.o(.TRACE)
    format                                   0x08804cdc   Data          48  key_handle.o(.TRACE)
    __tagsym$$used                           0x08804d0c   Number         0  key_handle.o(.TRACE)
    format                                   0x08804d0c   Data          70  key_handle.o(.TRACE)
    __tagsym$$used                           0x08804d54   Number         0  key_handle.o(.TRACE)
    format                                   0x08804d54   Data          48  key_handle.o(.TRACE)
    .TRACE                                   0x08804d84   Section      270  voice_driver.o(.TRACE)
    __tagsym$$used                           0x08804d84   Number         0  voice_driver.o(.TRACE)
    format                                   0x08804d84   Data          57  voice_driver.o(.TRACE)
    __tagsym$$used                           0x08804dc0   Number         0  voice_driver.o(.TRACE)
    format                                   0x08804dc0   Data          38  voice_driver.o(.TRACE)
    __tagsym$$used                           0x08804de8   Number         0  voice_driver.o(.TRACE)
    format                                   0x08804de8   Data          58  voice_driver.o(.TRACE)
    __tagsym$$used                           0x08804e24   Number         0  voice_driver.o(.TRACE)
    format                                   0x08804e24   Data          48  voice_driver.o(.TRACE)
    __tagsym$$used                           0x08804e54   Number         0  voice_driver.o(.TRACE)
    format                                   0x08804e54   Data          62  voice_driver.o(.TRACE)
    .TRACE                                   0x08804e94   Section     3327  voice.o(.TRACE)
    __tagsym$$used                           0x08804e94   Number         0  voice.o(.TRACE)
    format                                   0x08804e94   Data          38  voice.o(.TRACE)
    __tagsym$$used                           0x08804ebc   Number         0  voice.o(.TRACE)
    format                                   0x08804ebc   Data          62  voice.o(.TRACE)
    __tagsym$$used                           0x08804efc   Number         0  voice.o(.TRACE)
    format                                   0x08804efc   Data          50  voice.o(.TRACE)
    __tagsym$$used                           0x08804f30   Number         0  voice.o(.TRACE)
    format                                   0x08804f30   Data          66  voice.o(.TRACE)
    __tagsym$$used                           0x08804f74   Number         0  voice.o(.TRACE)
    format                                   0x08804f74   Data          89  voice.o(.TRACE)
    __tagsym$$used                           0x08804fd0   Number         0  voice.o(.TRACE)
    format                                   0x08804fd0   Data          54  voice.o(.TRACE)
    __tagsym$$used                           0x08805008   Number         0  voice.o(.TRACE)
    format                                   0x08805008   Data          62  voice.o(.TRACE)
    __tagsym$$used                           0x08805048   Number         0  voice.o(.TRACE)
    format                                   0x08805048   Data          49  voice.o(.TRACE)
    __tagsym$$used                           0x0880507c   Number         0  voice.o(.TRACE)
    format                                   0x0880507c   Data          56  voice.o(.TRACE)
    __tagsym$$used                           0x088050b4   Number         0  voice.o(.TRACE)
    format                                   0x088050b4   Data          60  voice.o(.TRACE)
    __tagsym$$used                           0x088050f0   Number         0  voice.o(.TRACE)
    format                                   0x088050f0   Data          59  voice.o(.TRACE)
    __tagsym$$used                           0x0880512c   Number         0  voice.o(.TRACE)
    format                                   0x0880512c   Data          67  voice.o(.TRACE)
    __tagsym$$used                           0x08805170   Number         0  voice.o(.TRACE)
    format                                   0x08805170   Data          45  voice.o(.TRACE)
    __tagsym$$used                           0x088051a0   Number         0  voice.o(.TRACE)
    format                                   0x088051a0   Data          47  voice.o(.TRACE)
    __tagsym$$used                           0x088051d0   Number         0  voice.o(.TRACE)
    format                                   0x088051d0   Data          43  voice.o(.TRACE)
    __tagsym$$used                           0x088051fc   Number         0  voice.o(.TRACE)
    format                                   0x088051fc   Data          69  voice.o(.TRACE)
    __tagsym$$used                           0x08805244   Number         0  voice.o(.TRACE)
    format                                   0x08805244   Data          83  voice.o(.TRACE)
    __tagsym$$used                           0x08805298   Number         0  voice.o(.TRACE)
    format                                   0x08805298   Data          68  voice.o(.TRACE)
    __tagsym$$used                           0x088052dc   Number         0  voice.o(.TRACE)
    format                                   0x088052dc   Data          70  voice.o(.TRACE)
    __tagsym$$used                           0x08805324   Number         0  voice.o(.TRACE)
    format                                   0x08805324   Data          64  voice.o(.TRACE)
    __tagsym$$used                           0x08805364   Number         0  voice.o(.TRACE)
    format                                   0x08805364   Data          43  voice.o(.TRACE)
    __tagsym$$used                           0x08805390   Number         0  voice.o(.TRACE)
    format                                   0x08805390   Data          78  voice.o(.TRACE)
    __tagsym$$used                           0x088053e0   Number         0  voice.o(.TRACE)
    format                                   0x088053e0   Data          57  voice.o(.TRACE)
    __tagsym$$used                           0x0880541c   Number         0  voice.o(.TRACE)
    format                                   0x0880541c   Data          77  voice.o(.TRACE)
    __tagsym$$used                           0x0880546c   Number         0  voice.o(.TRACE)
    format                                   0x0880546c   Data          70  voice.o(.TRACE)
    __tagsym$$used                           0x088054b4   Number         0  voice.o(.TRACE)
    format                                   0x088054b4   Data          76  voice.o(.TRACE)
    __tagsym$$used                           0x08805500   Number         0  voice.o(.TRACE)
    format                                   0x08805500   Data          75  voice.o(.TRACE)
    __tagsym$$used                           0x0880554c   Number         0  voice.o(.TRACE)
    format                                   0x0880554c   Data          70  voice.o(.TRACE)
    __tagsym$$used                           0x08805594   Number         0  voice.o(.TRACE)
    format                                   0x08805594   Data          83  voice.o(.TRACE)
    __tagsym$$used                           0x088055e8   Number         0  voice.o(.TRACE)
    format                                   0x088055e8   Data          59  voice.o(.TRACE)
    __tagsym$$used                           0x08805624   Number         0  voice.o(.TRACE)
    format                                   0x08805624   Data          74  voice.o(.TRACE)
    __tagsym$$used                           0x08805670   Number         0  voice.o(.TRACE)
    format                                   0x08805670   Data          52  voice.o(.TRACE)
    __tagsym$$used                           0x088056a4   Number         0  voice.o(.TRACE)
    format                                   0x088056a4   Data          76  voice.o(.TRACE)
    __tagsym$$used                           0x088056f0   Number         0  voice.o(.TRACE)
    format                                   0x088056f0   Data          42  voice.o(.TRACE)
    __tagsym$$used                           0x0880571c   Number         0  voice.o(.TRACE)
    format                                   0x0880571c   Data          45  voice.o(.TRACE)
    __tagsym$$used                           0x0880574c   Number         0  voice.o(.TRACE)
    format                                   0x0880574c   Data          57  voice.o(.TRACE)
    __tagsym$$used                           0x08805788   Number         0  voice.o(.TRACE)
    format                                   0x08805788   Data          58  voice.o(.TRACE)
    __tagsym$$used                           0x088057c4   Number         0  voice.o(.TRACE)
    format                                   0x088057c4   Data          85  voice.o(.TRACE)
    __tagsym$$used                           0x0880581c   Number         0  voice.o(.TRACE)
    format                                   0x0880581c   Data          47  voice.o(.TRACE)
    __tagsym$$used                           0x0880584c   Number         0  voice.o(.TRACE)
    format                                   0x0880584c   Data          71  voice.o(.TRACE)
    __tagsym$$used                           0x08805894   Number         0  voice.o(.TRACE)
    format                                   0x08805894   Data          68  voice.o(.TRACE)
    __tagsym$$used                           0x088058d8   Number         0  voice.o(.TRACE)
    format                                   0x088058d8   Data          92  voice.o(.TRACE)
    __tagsym$$used                           0x08805934   Number         0  voice.o(.TRACE)
    format                                   0x08805934   Data          68  voice.o(.TRACE)
    __tagsym$$used                           0x08805978   Number         0  voice.o(.TRACE)
    format                                   0x08805978   Data          53  voice.o(.TRACE)
    __tagsym$$used                           0x088059b0   Number         0  voice.o(.TRACE)
    format                                   0x088059b0   Data         112  voice.o(.TRACE)
    __tagsym$$used                           0x08805a20   Number         0  voice.o(.TRACE)
    format                                   0x08805a20   Data          72  voice.o(.TRACE)
    __tagsym$$used                           0x08805a68   Number         0  voice.o(.TRACE)
    format                                   0x08805a68   Data          54  voice.o(.TRACE)
    __tagsym$$used                           0x08805aa0   Number         0  voice.o(.TRACE)
    format                                   0x08805aa0   Data          66  voice.o(.TRACE)
    __tagsym$$used                           0x08805ae4   Number         0  voice.o(.TRACE)
    format                                   0x08805ae4   Data          51  voice.o(.TRACE)
    __tagsym$$used                           0x08805b18   Number         0  voice.o(.TRACE)
    format                                   0x08805b18   Data          66  voice.o(.TRACE)
    __tagsym$$used                           0x08805b5c   Number         0  voice.o(.TRACE)
    format                                   0x08805b5c   Data          55  voice.o(.TRACE)
    .TRACE                                   0x08805b94   Section      830  ir_send_driver.o(.TRACE)
    __tagsym$$used                           0x08805b94   Number         0  ir_send_driver.o(.TRACE)
    format                                   0x08805b94   Data          24  ir_send_driver.o(.TRACE)
    __tagsym$$used                           0x08805bac   Number         0  ir_send_driver.o(.TRACE)
    format                                   0x08805bac   Data          61  ir_send_driver.o(.TRACE)
    __tagsym$$used                           0x08805bec   Number         0  ir_send_driver.o(.TRACE)
    format                                   0x08805bec   Data          36  ir_send_driver.o(.TRACE)
    __tagsym$$used                           0x08805c10   Number         0  ir_send_driver.o(.TRACE)
    format                                   0x08805c10   Data          61  ir_send_driver.o(.TRACE)
    __tagsym$$used                           0x08805c50   Number         0  ir_send_driver.o(.TRACE)
    format                                   0x08805c50   Data          70  ir_send_driver.o(.TRACE)
    __tagsym$$used                           0x08805c98   Number         0  ir_send_driver.o(.TRACE)
    format                                   0x08805c98   Data          31  ir_send_driver.o(.TRACE)
    __tagsym$$used                           0x08805cb8   Number         0  ir_send_driver.o(.TRACE)
    format                                   0x08805cb8   Data          55  ir_send_driver.o(.TRACE)
    __tagsym$$used                           0x08805cf0   Number         0  ir_send_driver.o(.TRACE)
    format                                   0x08805cf0   Data          48  ir_send_driver.o(.TRACE)
    __tagsym$$used                           0x08805d20   Number         0  ir_send_driver.o(.TRACE)
    format                                   0x08805d20   Data          35  ir_send_driver.o(.TRACE)
    __tagsym$$used                           0x08805d44   Number         0  ir_send_driver.o(.TRACE)
    format                                   0x08805d44   Data          40  ir_send_driver.o(.TRACE)
    __tagsym$$used                           0x08805d6c   Number         0  ir_send_driver.o(.TRACE)
    format                                   0x08805d6c   Data          58  ir_send_driver.o(.TRACE)
    __tagsym$$used                           0x08805da8   Number         0  ir_send_driver.o(.TRACE)
    format                                   0x08805da8   Data          68  ir_send_driver.o(.TRACE)
    __tagsym$$used                           0x08805dec   Number         0  ir_send_driver.o(.TRACE)
    format                                   0x08805dec   Data          57  ir_send_driver.o(.TRACE)
    __tagsym$$used                           0x08805e28   Number         0  ir_send_driver.o(.TRACE)
    format                                   0x08805e28   Data          37  ir_send_driver.o(.TRACE)
    __tagsym$$used                           0x08805e50   Number         0  ir_send_driver.o(.TRACE)
    format                                   0x08805e50   Data          50  ir_send_driver.o(.TRACE)
    __tagsym$$used                           0x08805e84   Number         0  ir_send_driver.o(.TRACE)
    format                                   0x08805e84   Data          54  ir_send_driver.o(.TRACE)
    __tagsym$$used                           0x08805ebc   Number         0  ir_send_driver.o(.TRACE)
    format                                   0x08805ebc   Data          22  ir_send_driver.o(.TRACE)
    .TRACE                                   0x08805ed4   Section      581  ir_send_handle.o(.TRACE)
    __tagsym$$used                           0x08805ed4   Number         0  ir_send_handle.o(.TRACE)
    format                                   0x08805ed4   Data          53  ir_send_handle.o(.TRACE)
    __tagsym$$used                           0x08805f0c   Number         0  ir_send_handle.o(.TRACE)
    format                                   0x08805f0c   Data          91  ir_send_handle.o(.TRACE)
    __tagsym$$used                           0x08805f68   Number         0  ir_send_handle.o(.TRACE)
    format                                   0x08805f68   Data          87  ir_send_handle.o(.TRACE)
    __tagsym$$used                           0x08805fc0   Number         0  ir_send_handle.o(.TRACE)
    format                                   0x08805fc0   Data          74  ir_send_handle.o(.TRACE)
    __tagsym$$used                           0x0880600c   Number         0  ir_send_handle.o(.TRACE)
    format                                   0x0880600c   Data          56  ir_send_handle.o(.TRACE)
    __tagsym$$used                           0x08806044   Number         0  ir_send_handle.o(.TRACE)
    format                                   0x08806044   Data          59  ir_send_handle.o(.TRACE)
    __tagsym$$used                           0x08806080   Number         0  ir_send_handle.o(.TRACE)
    format                                   0x08806080   Data          60  ir_send_handle.o(.TRACE)
    __tagsym$$used                           0x088060bc   Number         0  ir_send_handle.o(.TRACE)
    format                                   0x088060bc   Data          63  ir_send_handle.o(.TRACE)
    __tagsym$$used                           0x088060fc   Number         0  ir_send_handle.o(.TRACE)
    format                                   0x088060fc   Data          29  ir_send_handle.o(.TRACE)
    .TRACE                                   0x0880611c   Section     2046  ir_service_handle.o(.TRACE)
    __tagsym$$used                           0x0880611c   Number         0  ir_service_handle.o(.TRACE)
    format                                   0x0880611c   Data          54  ir_service_handle.o(.TRACE)
    __tagsym$$used                           0x08806154   Number         0  ir_service_handle.o(.TRACE)
    format                                   0x08806154   Data          59  ir_service_handle.o(.TRACE)
    __tagsym$$used                           0x08806190   Number         0  ir_service_handle.o(.TRACE)
    format                                   0x08806190   Data          93  ir_service_handle.o(.TRACE)
    __tagsym$$used                           0x088061f0   Number         0  ir_service_handle.o(.TRACE)
    format                                   0x088061f0   Data          88  ir_service_handle.o(.TRACE)
    __tagsym$$used                           0x08806248   Number         0  ir_service_handle.o(.TRACE)
    format                                   0x08806248   Data          80  ir_service_handle.o(.TRACE)
    __tagsym$$used                           0x08806298   Number         0  ir_service_handle.o(.TRACE)
    format                                   0x08806298   Data          94  ir_service_handle.o(.TRACE)
    __tagsym$$used                           0x088062f8   Number         0  ir_service_handle.o(.TRACE)
    format                                   0x088062f8   Data          90  ir_service_handle.o(.TRACE)
    __tagsym$$used                           0x08806354   Number         0  ir_service_handle.o(.TRACE)
    format                                   0x08806354   Data          68  ir_service_handle.o(.TRACE)
    __tagsym$$used                           0x08806398   Number         0  ir_service_handle.o(.TRACE)
    format                                   0x08806398   Data          90  ir_service_handle.o(.TRACE)
    __tagsym$$used                           0x088063f4   Number         0  ir_service_handle.o(.TRACE)
    format                                   0x088063f4   Data          38  ir_service_handle.o(.TRACE)
    __tagsym$$used                           0x0880641c   Number         0  ir_service_handle.o(.TRACE)
    format                                   0x0880641c   Data          53  ir_service_handle.o(.TRACE)
    __tagsym$$used                           0x08806454   Number         0  ir_service_handle.o(.TRACE)
    format                                   0x08806454   Data          59  ir_service_handle.o(.TRACE)
    __tagsym$$used                           0x08806490   Number         0  ir_service_handle.o(.TRACE)
    format                                   0x08806490   Data         104  ir_service_handle.o(.TRACE)
    __tagsym$$used                           0x088064f8   Number         0  ir_service_handle.o(.TRACE)
    format                                   0x088064f8   Data          57  ir_service_handle.o(.TRACE)
    __tagsym$$used                           0x08806534   Number         0  ir_service_handle.o(.TRACE)
    format                                   0x08806534   Data          66  ir_service_handle.o(.TRACE)
    __tagsym$$used                           0x08806578   Number         0  ir_service_handle.o(.TRACE)
    format                                   0x08806578   Data          91  ir_service_handle.o(.TRACE)
    __tagsym$$used                           0x088065d4   Number         0  ir_service_handle.o(.TRACE)
    format                                   0x088065d4   Data          90  ir_service_handle.o(.TRACE)
    __tagsym$$used                           0x08806630   Number         0  ir_service_handle.o(.TRACE)
    format                                   0x08806630   Data          78  ir_service_handle.o(.TRACE)
    __tagsym$$used                           0x08806680   Number         0  ir_service_handle.o(.TRACE)
    format                                   0x08806680   Data          86  ir_service_handle.o(.TRACE)
    __tagsym$$used                           0x088066d8   Number         0  ir_service_handle.o(.TRACE)
    format                                   0x088066d8   Data          87  ir_service_handle.o(.TRACE)
    __tagsym$$used                           0x08806730   Number         0  ir_service_handle.o(.TRACE)
    format                                   0x08806730   Data          43  ir_service_handle.o(.TRACE)
    __tagsym$$used                           0x0880675c   Number         0  ir_service_handle.o(.TRACE)
    format                                   0x0880675c   Data          68  ir_service_handle.o(.TRACE)
    __tagsym$$used                           0x088067a0   Number         0  ir_service_handle.o(.TRACE)
    format                                   0x088067a0   Data          43  ir_service_handle.o(.TRACE)
    __tagsym$$used                           0x088067cc   Number         0  ir_service_handle.o(.TRACE)
    format                                   0x088067cc   Data          51  ir_service_handle.o(.TRACE)
    __tagsym$$used                           0x08806800   Number         0  ir_service_handle.o(.TRACE)
    format                                   0x08806800   Data          54  ir_service_handle.o(.TRACE)
    __tagsym$$used                           0x08806838   Number         0  ir_service_handle.o(.TRACE)
    format                                   0x08806838   Data          66  ir_service_handle.o(.TRACE)
    __tagsym$$used                           0x0880687c   Number         0  ir_service_handle.o(.TRACE)
    format                                   0x0880687c   Data          71  ir_service_handle.o(.TRACE)
    __tagsym$$used                           0x088068c4   Number         0  ir_service_handle.o(.TRACE)
    format                                   0x088068c4   Data          86  ir_service_handle.o(.TRACE)
    .TRACE                                   0x0880691c   Section       34  led_driver.o(.TRACE)
    __tagsym$$used                           0x0880691c   Number         0  led_driver.o(.TRACE)
    format                                   0x0880691c   Data          34  led_driver.o(.TRACE)
    .TRACE                                   0x08806940   Section      157  buzzer_driver.o(.TRACE)
    __tagsym$$used                           0x08806940   Number         0  buzzer_driver.o(.TRACE)
    format                                   0x08806940   Data          32  buzzer_driver.o(.TRACE)
    __tagsym$$used                           0x08806960   Number         0  buzzer_driver.o(.TRACE)
    format                                   0x08806960   Data          79  buzzer_driver.o(.TRACE)
    __tagsym$$used                           0x088069b0   Number         0  buzzer_driver.o(.TRACE)
    format                                   0x088069b0   Data          45  buzzer_driver.o(.TRACE)
    .TRACE                                   0x088069e0   Section      767  fms_service_handle.o(.TRACE)
    __tagsym$$used                           0x088069e0   Number         0  fms_service_handle.o(.TRACE)
    format                                   0x088069e0   Data          47  fms_service_handle.o(.TRACE)
    __tagsym$$used                           0x08806a10   Number         0  fms_service_handle.o(.TRACE)
    format                                   0x08806a10   Data          52  fms_service_handle.o(.TRACE)
    __tagsym$$used                           0x08806a44   Number         0  fms_service_handle.o(.TRACE)
    format                                   0x08806a44   Data          86  fms_service_handle.o(.TRACE)
    __tagsym$$used                           0x08806a9c   Number         0  fms_service_handle.o(.TRACE)
    format                                   0x08806a9c   Data          77  fms_service_handle.o(.TRACE)
    __tagsym$$used                           0x08806aec   Number         0  fms_service_handle.o(.TRACE)
    format                                   0x08806aec   Data          69  fms_service_handle.o(.TRACE)
    __tagsym$$used                           0x08806b34   Number         0  fms_service_handle.o(.TRACE)
    format                                   0x08806b34   Data          36  fms_service_handle.o(.TRACE)
    __tagsym$$used                           0x08806b58   Number         0  fms_service_handle.o(.TRACE)
    format                                   0x08806b58   Data          36  fms_service_handle.o(.TRACE)
    __tagsym$$used                           0x08806b7c   Number         0  fms_service_handle.o(.TRACE)
    format                                   0x08806b7c   Data          44  fms_service_handle.o(.TRACE)
    __tagsym$$used                           0x08806ba8   Number         0  fms_service_handle.o(.TRACE)
    format                                   0x08806ba8   Data          78  fms_service_handle.o(.TRACE)
    __tagsym$$used                           0x08806bf8   Number         0  fms_service_handle.o(.TRACE)
    format                                   0x08806bf8   Data          41  fms_service_handle.o(.TRACE)
    __tagsym$$used                           0x08806c24   Number         0  fms_service_handle.o(.TRACE)
    format                                   0x08806c24   Data          80  fms_service_handle.o(.TRACE)
    __tagsym$$used                           0x08806c74   Number         0  fms_service_handle.o(.TRACE)
    format                                   0x08806c74   Data          38  fms_service_handle.o(.TRACE)
    __tagsym$$used                           0x08806c9c   Number         0  fms_service_handle.o(.TRACE)
    format                                   0x08806c9c   Data          67  fms_service_handle.o(.TRACE)
    .TRACE                                   0x08806ce0   Section     1197  battery_driver.o(.TRACE)
    __tagsym$$used                           0x08806ce0   Number         0  battery_driver.o(.TRACE)
    format                                   0x08806ce0   Data          62  battery_driver.o(.TRACE)
    __tagsym$$used                           0x08806d20   Number         0  battery_driver.o(.TRACE)
    format                                   0x08806d20   Data          41  battery_driver.o(.TRACE)
    __tagsym$$used                           0x08806d4c   Number         0  battery_driver.o(.TRACE)
    format                                   0x08806d4c   Data          59  battery_driver.o(.TRACE)
    __tagsym$$used                           0x08806d88   Number         0  battery_driver.o(.TRACE)
    format                                   0x08806d88   Data          55  battery_driver.o(.TRACE)
    __tagsym$$used                           0x08806dc0   Number         0  battery_driver.o(.TRACE)
    format                                   0x08806dc0   Data          59  battery_driver.o(.TRACE)
    __tagsym$$used                           0x08806dfc   Number         0  battery_driver.o(.TRACE)
    format                                   0x08806dfc   Data          54  battery_driver.o(.TRACE)
    __tagsym$$used                           0x08806e34   Number         0  battery_driver.o(.TRACE)
    format                                   0x08806e34   Data          52  battery_driver.o(.TRACE)
    __tagsym$$used                           0x08806e68   Number         0  battery_driver.o(.TRACE)
    format                                   0x08806e68   Data          57  battery_driver.o(.TRACE)
    __tagsym$$used                           0x08806ea4   Number         0  battery_driver.o(.TRACE)
    format                                   0x08806ea4   Data          53  battery_driver.o(.TRACE)
    __tagsym$$used                           0x08806edc   Number         0  battery_driver.o(.TRACE)
    format                                   0x08806edc   Data          54  battery_driver.o(.TRACE)
    __tagsym$$used                           0x08806f14   Number         0  battery_driver.o(.TRACE)
    format                                   0x08806f14   Data          29  battery_driver.o(.TRACE)
    __tagsym$$used                           0x08806f34   Number         0  battery_driver.o(.TRACE)
    format                                   0x08806f34   Data          46  battery_driver.o(.TRACE)
    __tagsym$$used                           0x08806f64   Number         0  battery_driver.o(.TRACE)
    format                                   0x08806f64   Data          30  battery_driver.o(.TRACE)
    __tagsym$$used                           0x08806f84   Number         0  battery_driver.o(.TRACE)
    format                                   0x08806f84   Data          55  battery_driver.o(.TRACE)
    __tagsym$$used                           0x08806fbc   Number         0  battery_driver.o(.TRACE)
    format                                   0x08806fbc   Data          63  battery_driver.o(.TRACE)
    __tagsym$$used                           0x08806ffc   Number         0  battery_driver.o(.TRACE)
    format                                   0x08806ffc   Data          49  battery_driver.o(.TRACE)
    __tagsym$$used                           0x08807030   Number         0  battery_driver.o(.TRACE)
    format                                   0x08807030   Data          48  battery_driver.o(.TRACE)
    __tagsym$$used                           0x08807060   Number         0  battery_driver.o(.TRACE)
    format                                   0x08807060   Data          45  battery_driver.o(.TRACE)
    __tagsym$$used                           0x08807090   Number         0  battery_driver.o(.TRACE)
    format                                   0x08807090   Data          49  battery_driver.o(.TRACE)
    __tagsym$$used                           0x088070c4   Number         0  battery_driver.o(.TRACE)
    format                                   0x088070c4   Data         110  battery_driver.o(.TRACE)
    __tagsym$$used                           0x08807134   Number         0  battery_driver.o(.TRACE)
    format                                   0x08807134   Data          47  battery_driver.o(.TRACE)
    __tagsym$$used                           0x08807164   Number         0  battery_driver.o(.TRACE)
    format                                   0x08807164   Data          41  battery_driver.o(.TRACE)
    .TRACE                                   0x08807190   Section        6  frm_vpk_log.o(.TRACE)
    __tagsym$$used                           0x08807190   Number         0  frm_vpk_log.o(.TRACE)
    format                                   0x08807190   Data           6  frm_vpk_log.o(.TRACE)

    Global Symbols

    Symbol Name                              Value     Ov Type        Size  Object(Section)

    BuildAttributes$$THM_ISAv3M$S$PE$A:L22$X:L11$S22$IEEE1$IW$USESV6$~STKCKD$USESV7$~SHL$OTIME$ROPI$IEEEJ$EBA8$UX$STANDARDLIB$REQ8$PRES8$EABIv2 0x00000000   Number         0  anon$$obj.o ABSOLUTE
    Image$$CACHE_DATA_ON$$RO$$Length         0x00000000   Number         0  anon$$obj.o ABSOLUTE
    Image$$CACHE_DATA_ON$$RW$$Length         0x00000000   Number         0  anon$$obj.o ABSOLUTE
    Image$$CACHE_DATA_ON$$ZI$$Length         0x00000000   Number         0  anon$$obj.o ABSOLUTE
    Image$$OVERLAY_A$$RW$$Length             0x00000000   Number         0  anon$$obj.o ABSOLUTE
    Image$$OVERLAY_A$$ZI$$Length             0x00000000   Number         0  anon$$obj.o ABSOLUTE
    Image$$OVERLAY_B$$RO$$Length             0x00000000   Number         0  anon$$obj.o ABSOLUTE
    Image$$OVERLAY_B$$RW$$Length             0x00000000   Number         0  anon$$obj.o ABSOLUTE
    Image$$OVERLAY_B$$ZI$$Length             0x00000000   Number         0  anon$$obj.o ABSOLUTE
    Image$$OVERLAY_C$$RO$$Length             0x00000000   Number         0  anon$$obj.o ABSOLUTE
    Image$$OVERLAY_C$$RW$$Length             0x00000000   Number         0  anon$$obj.o ABSOLUTE
    Image$$OVERLAY_C$$ZI$$Length             0x00000000   Number         0  anon$$obj.o ABSOLUTE
    __ARM_use_no_argv                        0x00000000   Number         0  main.o ABSOLUTE
    _printf_flags                            0x00000000   Number         0  printf_stubs.o ABSOLUTE
    _printf_return_value                     0x00000000   Number         0  printf_stubs.o ABSOLUTE
    _printf_sizespec                         0x00000000   Number         0  printf_stubs.o ABSOLUTE
    _printf_widthprec                        0x00000000   Number         0  printf_stubs.o ABSOLUTE
    __ARM_exceptions_init                     - Undefined Weak Reference
    __alloca_initialize                       - Undefined Weak Reference
    __arm_preinit_                            - Undefined Weak Reference
    __cpp_initialize__aeabi_                  - Undefined Weak Reference
    __scatterload                             - Undefined Weak Reference
    __sigvec_lookup                           - Undefined Weak Reference
    _atexit_init                              - Undefined Weak Reference
    _clock_init                               - Undefined Weak Reference
    _fp_trap_init                             - Undefined Weak Reference
    _get_lc_collate                           - Undefined Weak Reference
    _get_lc_monetary                          - Undefined Weak Reference
    _get_lc_time                              - Undefined Weak Reference
    _getenv_init                              - Undefined Weak Reference
    _handle_redirection                       - Undefined Weak Reference
    _init_alloc                               - Undefined Weak Reference
    _init_user_alloc                          - Undefined Weak Reference
    _initio                                   - Undefined Weak Reference
    _printf_mbtowc                            - Undefined Weak Reference
    _printf_wc                                - Undefined Weak Reference
    _signal_init                              - Undefined Weak Reference
    Image$$OVERLAY_A$$RO$$Length             0x000000c8   Number         0  anon$$obj.o ABSOLUTE
    Image$$RAM_VECTOR_TABLE$$RO$$Length      0x000000e8   Number         0  anon$$obj.o ABSOLUTE
    __Vectors_Size                           0x000000e8   Number         0  startup_rtl876x.o ABSOLUTE
    vAssertHandler                           0x00000209   Thumb Code     0  ROM.lib ABSOLUTE
    WDG_SystemReset                          0x0000029d   Thumb Code     0  ROM.lib ABSOLUTE
    __aeabi_memcpy4                          0x000002a9   Thumb Code     0  ROM.lib ABSOLUTE
    __aeabi_memcpy8                          0x000002a9   Thumb Code     0  ROM.lib ABSOLUTE
    Image$$RAM_DATA_ON$$RW$$Length           0x000003b0   Number         0  anon$$obj.o ABSOLUTE
    Image$$RAM_DATA_ON$$RO$$Length           0x000014a8   Number         0  anon$$obj.o ABSOLUTE
    Image$$RAM_DATA_ON$$ZI$$Length           0x000025ac   Number         0  anon$$obj.o ABSOLUTE
    RamVectorTableInit                       0x000034d1   Thumb Code     0  ROM.lib ABSOLUTE
    RamVectorTableUpdate                     0x000034f7   Thumb Code     0  ROM.lib ABSOLUTE
    LOGUARTDriverInit                        0x000037ed   Thumb Code     0  ROM.lib ABSOLUTE
    DumpRawMemory                            0x000043ab   Thumb Code     0  ROM.lib ABSOLUTE
    dump_raw_memory_all                      0x00004519   Thumb Code     0  ROM.lib ABSOLUTE
    hardfault_print_buffered_log             0x00004573   Thumb Code     0  ROM.lib ABSOLUTE
    ROM_Default_Handler                      0x000047e7   Thumb Code     0  ROM.lib ABSOLUTE
    SystemCall                               0x0000491b   Thumb Code     0  ROM.lib ABSOLUTE
